:04000000FCEF26F0FB
:1000080000C019F001C018F00BC017F00CC016F0B2
:100018000DC015F0E1CF1AF0E2CF1BF001015A89AB
:100028009EAA65D09DAA63D0F1EC17F000C0F9F242
:10003800ABA20FD0AB98010E01015825006E000E3F
:100048005921016E00C058F101C059F1AB88020175
:10005800F96BABA411D0AB9E010E01015825006EBF
:10006800000E5921016E00C058F101C059F1AB8E44
:10007800F1EC17F000C0F9F20201F9510D0A08E09D
:1000880003010251000802E101517F0801E315D084
:10009800010E0201FE6F000EFF6FFF0E0301012526
:1000A800E16E010E0221E26EE66A9D9A01C38CF2AE
:1000B80002C38DF2016B026B1AD00201FE6BFF6B5B
:1000C800FF0E03010125E16E010E0221E26EF9C265
:1000D800E6FF01C38CF202C38DF2010E0125006E0A
:1000E800000E0221016E00C001F301C002F3F2A864
:1000F80015D0F2A213D0F298010E0001E56F000EA0
:10010800E66F030E0B6E080E0C6E770E0D6E0D2E3D
:10011800FED70C2EFCD70B2EFAD7F292F2AA07D0F4
:10012800F2A405D0D59EF29A010E5F6EF29419C022
:1001380000F018C001F017C00BF016C00CF015C085
:0C0148000DF01AC0E1FF1BC0E2FF110027
:0C01540072B201D0FDD741C373FF12004E
:0E016000ACB202D00000FCD741C3ADFF1200CC
:10016E0003014151030A00E14151040A00E14151EA
:0C017E00050A00E14151060A00E11200F0
:10018A00F250026EF29E0500FF6A0150FE6E0050A8
:08019A00FD6E02BEF28E1200A0
:1001A200C7B409D01F0EC514016E0150000A03E145
:0A01B200010E006E01D0006A120079
:0401BC00C5841200E4
:1001C0009E963BC3C9FF71C03CF372C03DF373C040
:1001D0003EF374C03FF3C7A422D0000171517211E5
:1001E000731174111BE003013C513D113E113F118D
:1001F0000EE144C1E1FF45C1E2FF040EE66E42C1DB
:1002000000F043C101F0C1DF010E006E3BD0010ED2
:1002100003013C5F000E3D5B3E5B3F5BDCD771C082
:100220003CF372C03DF373C03EF374C03FF39EB61F
:1002300022D0000171517211731174111BE003017E
:100240003C513D113E113F110EE144C1E1FF45C15A
:10025000E2FF040EE66E42C100F043C101F095DFFB
:10026000010E006E0FD0010E03013C5F000E3D5BDE
:100270003E5B3F5BDCD7C5BC02D0006A03D0C584BF
:06028000020E006E1200E8
:1002860071C03DF372C03EF373C03FF374C040F3D8
:1002960003013B6B3C6B3C51120802E13B518E085B
:1002A60008E37CDF005201E004D003013B4B3C2B0A
:1002B600F2D70301120E3C5D02E18F0E3B5D03E3B4
:1002C6007B0E006E26D0C580C5A022D000017151DC
:1002D6007211731174111BE003013D513E113F1160
:1002E60040110EE144C1E1FF45C1E2FF050EE66E95
:1002F60042C100F043C101F045DF010E006E09D096
:10030600010E03013D5F000E3E5B3F5B405BDCD7A9
:04031600006A120067
:08031A000AAE029E000E120063
:100322000B840BAE9CEF01F0010E036E026A016AB0
:0A033200006A0A360232FF0E1200C4
:0E033C00026A016A006A086A036A000E120073
:10034A000B820BAEAFEF01F0036802680168006828
:08035A000A360232FF0E120008
:100362000CB0F3EF01F00CA299EF02F00E6A000E4E
:1003720002640AEF02F0F00E0214D8A4D5EF01F0E5
:10038200023A01380F0B02260138F00B016E0038D9
:100392000F0B01260038F00B006E08380F0B0026F9
:1003A2000838F00B086E0E84D89002BEEEEF01F012
:1003B20008360036013602360E2A02BEEEEF01F092
:1003C20008360036013602360E2A02BEEEEF01F082
:1003D20008360036013602360E2A0E5003648FEFBD
:1003E20002F0035E0BBC08AE94EF02F0D880800EE0
:1003F20008640030000E002201220222D8A094EFED
:1004020002F0023201320032034A99EF02F094EF15
:1004120002F001C002F000C001F008C000F0086A5A
:10042200000E0E86026441EF02F0F00E0214D8A410
:1004320029EF02F0023A01380F0B02260138F00BC5
:10044200016E00380F0B01260038F00B006E0E848F
:10045200D89002BEEEEF01F00036013602360E2AC7
:1004620002BEEEEF01F00036013602360E2A02BE5F
:10047200EEEF01F00036013602360E2AEEEF01F001
:1004820001C002F000C001F0006A000E0E960E8854
:1004920002646EEF02F0F00E0214D8A459EF02F0DB
:1004A200023A01380F0B02260138F00B016E0E845E
:1004B200D89002BEEEEF01F0013602360E2A02BEDD
:1004C200EEEF01F0013602360E2A02BEEEEF01F027
:1004D200013602360E2AEEEF01F001C002F0016A87
:1004E200000E0E8602649EEF02F0F00E0214D8A4F3
:1004F2007DEF02F0023A0E84D89002BEEEEF01F0D8
:1005020002360E2A02BEEEEF01F002360E2A02BEBB
:10051200EEEF01F002360E2AEEEF01F0010E0C6E44
:10052200FFDEA1EF02F0020E0C6EF6DEA1EF02F08A
:10053200040E0C6E09DFA1EF02F0080E0C6EFDDE58
:020542001200A5
:10054400A0DE38C33BF33ADE00C03AF3000E016E7E
:10055400FF0E011802E1FF0E001803E1C9CF7FF27C
:10056400C69E39C33BF32ADE00C03AF325DE3AC304
:0405740000F0120081
:100578000B800BAEC8EF02F0026A0AAEFF0E026EE5
:0C058800016E006E0A360232FF0E1200F7
:0C0594003A0E0D6E0D2EFED70000120076
:0805A0000B6A0B86FF0E12002E
:1005A800086A096A100E0C6E0134083609360450C0
:1005B800085E0550D8A0053C095ED8B007D00450A5
:1005C80008260550D8B0053C0926D89000360136D3
:0605D8000C2EEAD7120010
:1005DE00F00E03013215006E008600C080F260C07E
:1005EE0038F3040E0010396FA6DF00C07FF20D0E37
:1005FE000D6E0D2EFED760C038F3FB0E0201801576
:10060E000301396F98DF00C07FF20D0E0D6E0D2EB7
:10061E00FED732C300F00036009000360090003650
:10062E00009000360090F00E0016008600C080F29A
:10063E0060C038F3040E00100301396F7CDF00C078
:10064E007FF2050E0D6E0D2EFED760C038F3FB0E39
:10065E00020180150301396F6EDF00C07FF2150EA7
:10066E000C6EC60E0D6E0D2EFED70C2EFCD7000096
:02067E00120068
:10068000025006180E6E086A096A0B6A0350076466
:1006900033EF04F006500A6E068E028E03500B6E86
:1006A0000750036E000E0B6483EF03F00B50075EE0
:1006B000D8B424EF04F0070E0764F2EF03F0075EEE
:1006C00000C008F001C000F002C001F0026A074E4D
:1006D00024EF04F00764C7EF03F0075E00C008F0E2
:1006E00001C000F0016A074E24EF04F00764A5EF93
:1006F00003F0075E00C008F0006A074E24EF04F024
:1007000007648CEF03F00AC002F005C001F004C0DA
:1007100000F0086A4DEF05F0030E076497EF03F051
:10072000075E08380F0B086E074E24EF04F0D890D0
:100730000832074E24EF04F0D8900832074E24EF19
:1007400004F0D890083224EF04F0030E0764B6EFEB
:1007500003F0075E08380F0B086E0038F00B082610
:1007600000380F0B006E074E24EF04F0D8900032D3
:100770000832074E24EF04F0D89000320832074EBA
:1007800024EF04F0D8900032083224EF04F0030E76
:100790000764DEEF03F0075E08380F0B086E0038C1
:1007A000F00B082600380F0B006E0138F00B002606
:1007B00001380F0B016E074E24EF04F0D890013280
:1007C00000320832074E24EF04F0D8900132003294
:1007D0000832074E24EF04F0D8900132003208327C
:1007E00024EF04F0030E07640FEF04F0075E0838EF
:1007F0000F0B086E0038F00B082600380F0B006E48
:100800000138F00B002601380F0B016E0238F00B97
:10081000012602380F0B026E074E24EF04F0D89029
:100820000232013200320832074E24EF04F0D89031
:100830000232013200320832074E24EF04F0D89021
:100840000232013200320832096A000E0EAE18EF91
:1008500005F0081E001E011E021E082A00220122A9
:10086000022218EF05F00750D8A439EF04F04DEF3D
:1008700005F0096A02C00AF0028E068E0750035C7A
:10088000076ED8B40BEF05F0070E0764D9EF04F03C
:10089000075E0450096E0550046E0650056E066A28
:1008A000074E0BEF05F0070E0764AEEF04F0075E8E
:1008B0000450096E0550046E056A074E0BEF05F0F3
:1008C000070E07648CEF04F0075E0450096E046A9B
:1008D000074E0BEF05F0070E076473EF04F00AC034
:1008E00002F04DEF05F0030E07647EEF04F0075EA3
:1008F00009380F0B096E074E0BEF05F0D89009323F
:10090000074E0BEF05F0D8900932074E0BEF05F0BC
:10091000D89009320BEF05F0030E07649DEF04F049
:10092000075E09380F0B096E0438F00B09260438EE
:100930000F0B046E074E0BEF05F0D890043209320E
:10094000074E0BEF05F0D89004320932074E0BEF3B
:1009500005F0D890043209320BEF05F0030E07645E
:10096000C5EF04F0075E09380F0B096E0438F00B71
:10097000092604380F0B046E0538F00B04260538E1
:100980000F0B056E074E0BEF05F0D89005320432C1
:100990000932074E0BEF05F0D890053204320932C8
:1009A000074E0BEF05F0D8900532043209320BEFF9
:1009B00005F0030E0764F6EF04F0075E09380F0B2D
:1009C000096E0438F00B092604380F0B046E053845
:1009D000F00B042605380F0B056E0638F00B0526C4
:1009E00006380F0B066E074E0BEF05F0D890063257
:1009F000053204320932074E0BEF05F0D89006326B
:100A0000053204320932074E0BEF05F0D89006325A
:100A1000053204320932086A000E0EAE18EF05F0F6
:100A2000091E041E051E061E092A0422052206228E
:100A300009500826045000220550012206500222C7
:100A40000EBE2FEF05F0D8A03EEF05F002320132C6
:100A500000320832033E3EEF05F048EF05F0D8B013
:100A600043EF05F0000E081E001E011E021E082A9C
:100A70000022012202220A7E43EF05F0010E0C6ED5
:100A800070DC4FEF05F0020E0C6E6BDC4FEF05F0E3
:100A9000040E0C6E5ADC4FEF05F0000E0C6E1200C7
:100AA0000C6A0E6A0250D8A469EF05F001C002F08A
:100AB00000C001F0006A0E860250D8A469EF05F06C
:100AC00001C002F0016A0E960E880250D8B47BEF86
:100AD00005F00E50035ED8A4D8A080EF05F0D890A2
:100AE00002BE85EF05F0003601360236032E70EFA8
:100AF00005F080EF05F0010E0C6E20DC88EF05F0AC
:100B0000020E0C6E0EDC88EF05F0040E0C6E05DC98
:020B10001200D1
:100B1200F00E03013215006E0086008000C080F2E4
:100B220060C038F3040E0010396F0BDD00C07FF295
:100B3200050E0D6E0D2EFED760C038F3FB0E0201BE
:100B420080150301396FFDDC00C07FF2050E0D6ECA
:100B52000D2EFED732C300F0003600900036009012
:100B62000036009000360090F00E001600860080DD
:100B720000C080F260C038F3040E00100301396F28
:100B8200E0DC00C07FF2050E0D6E0D2EFED760C0B8
:100B920038F3FB0E020180150301396FD2DC00C06D
:0C0BA2007FF2050E0D6E0D2EFED7120026
:100BAE0071C032F372C033F373C034F374C035F3D3
:100BBE00C582C5A221D00001715172117311741139
:100BCE001AE0030132513311341135110DE144C1D4
:100BDE00E1FF45C1E2FF060EE66E42C100F043C1E1
:100BEE0001F0C5EC00F008D0010E0301325F000EDB
:0A0BFE00335B345B355BDDD712007A
:100C080071C034F372C035F373C036F374C037F370
:100C18009E96C5869EB621D000017151721173113E
:100C280074111AE0030134513511361137110DE1F1
:100C380044C1E1FF45C1E2FF030EE66E42C100F088
:100C480043C101F0C5EC00F008D0010E0301345F88
:100C5800000E355B365B375BDDD70301C9CF33F355
:100C68003251000A02E1C58A01D0C59A9E96C5880C
:100C780071C034F372C035F373C036F374C037F300
:100C88009EB621D0000171517211731174111AE0CE
:100C9800030134513511361137110DE144C1E1FF1B
:100CA80045C1E2FF030EE66E42C100F043C101F008
:100CB800C5EC00F008D0010E0301345F000E355B6F
:0C0CC800365B375BDDD733C300F0120051
:100CD400086A080E0C6E003408360450085ED8B05A
:0E0CE40002D00826D89000360C2EF5D712004C
:100CF2000B6A0A6A096A00500402F4CF09F0F3CFC2
:100D020008F001500502F4CF0BF0F3CF0AF00050C7
:100D12000502F3500926F4500A22E86A0B22015018
:100D22000402F3500926F4500A22E86A0B2208C092
:100D320000F009C001F00AC002F00BC003F012007B
:100D420003013251390806E3300E325D03E3010E2E
:080D5200006E01D0006A1200DE
:100D5A000A6A0350D8A40A800750D8A40A820A5003
:100D6A00D8B410EF07F0030AD8B4C9EF06F00AB0F6
:100D7A00C4EF06F006AE0EEF07F00CEF07F002AE76
:100D8A000CEF07F00EEF07F00250800B0A6E029E7E
:100D9A000650800B069E0A18D8B4DAEF06F00A50FD
:100DAA00D8B40CEF07F00EEF07F00750035CD8B485
:100DBA00E4EF06F0D8A000EF07F006EF07F00650C0
:100DCA00025CD8B4EEEF06F0D8A000EF07F006EF09
:100DDA0007F00550015CD8B4F8EF06F0D8A000EF90
:100DEA0007F006EF07F00450005CD8B410EF07F0E4
:100DFA00D8B006EF07F00A52D8B40EEF07F00CEF9E
:100E0A0007F00A52D8B40CEF07F00EEF07F0D880BB
:0E0E1A001200D8901200D880D8841200120066
:100E2800A6A202D00000FCD7A69C2BC3AAFF2AC307
:100E3800A9FF2CC3A8FFA69EA684F2CF00F0F29EBD
:100E4800550EA76EAA0EA76EA68200BE02D0F29E0D
:100E580001D0F28EA694A1B802D00000FCD7A198C8
:020E6800120076
:100E6A002AC3F6FF2BC3F7FF2CC3F8FF0900F5CFFF
:100E7A0000F0005211E02AC3F6FF2BC3F7FF2CC380
:100E8A00F8FF0900F5CF32F33FDE010E03012A27EE
:0A0E9A00000E2B232C23E4D71200D6
:100EA4000D0E0301416FB0EC00F00A0E0301416F17
:060EB400B0EC00F012009A
:100EBA0003012C6B2D6B2AC303F02BC304F02AC346
:100ECA0005F02BC306F003C0E9FF04C0EAFFEE50A9
:100EDA00200A04E12C512D1101E110D0010E2C6FD2
:100EEA00000E2D6F03C0E9FF04C0EAFF05C0E1FF51
:100EFA0006C0E2FFEECFE6FF054A062A03C001F06C
:100F0A0004C002F0034A042A01C0E9FF02C0EAFF52
:100F1A00EE50000AD8E12AC300F02BC301F01200F8
:100F2A000201E26BE36B036A080E035C42E282B0E1
:100F3A000AD0E24BE32B000EE35D02E1C80EE25D4C
:100F4A0001E301D0F4D7850E0D6E0D2EFED782B0C7
:100F5A0011D003500708006E00C001F0010E006EA8
:100F6A00015004E000360090FF0FFBD7001E00502E
:100F7A0002161DD003500708006E00C001F0010ED2
:100F8A00006E015004E000360090FF0FFBD70050BE
:100F9A000212E26BE36B82A00AD0E24BE32B000E53
:100FAA00E35D02E1C80EE25D01E301D0F4D7032A52
:100FBA00BBD7010EE35D02E18F0EE25D07E3E2C2F9
:100FCA00E0F2E3C2E1F2E94BEA2B026A02C000F066
:020FDA00120003
:100FDC000450000A12E10550000A0FE10650000A05
:100FEC000CE10750000A09E1FF0E006EFF0E016EC6
:100FFC007F0E026EFF0E036EA8D0086A096A0750B6
:10100C00D8B499EF08F00350D8B49EEF08F0025012
:10101C0006180A6E028E068E0E6A02C008F001C017
:10102C000CF000C00DF004500D5E0550D8A0053C2E
:10103C000C5E0650D8A0063C085E086A0C6A0D6A65
:10104C00D8A030EF08F0D8900232013200320832CA
:10105C00010E0E6E0750035ED8A03DEF08F07E0E19
:10106C000E240326D8B0A3EF08F043EF08F07E0E51
:10107C000E240326D8A0A8EF08F0180E0B6E0D3620
:10108C000C3608360036013602360E360450005E39
:10109C000550D8A0053C015E0650D8A0063C025E67
:1010AC0006340E120EA05EEF08F00D8069EF08F00A
:1010BC00045000260550D8B0053C01260650D8B087
:1010CC00062802260D900B2E45EF08F08FEF08F046
:1010DC00D8900036013602360E360450005E0550AC
:1010EC00D8A0053C015E0650D8A0063C025E063432
:1010FC000E10010B0D26D8B00C2AD8B4082AD8A48F
:10110C008FEF08F008320C320D32032AD8B4A3EF5B
:10111C0008F00AAE089E0850026E0C50016E0D507D
:10112C00006EABEF08F0010ED0EC02F0ABEF08F064
:10113C00020E9EEC01F0ABEF08F0040EA5EC01F0F2
:0C114C00ABEF08F0080E91EC01F012006F
:10115800086A096A000E0762036431EF09F0025059
:1011680006180A6E075003267E0ED8A0C2EF08F0B4
:10117800035ED8B036EF09F0C6EF08F0035ED8A0DA
:101188003BEF09F0028E068E02C00EF001C00BF094
:1011980000C00DF000500402F4CF0CF0015005021D
:1011A800F4CF00F0F3CF08F00402F3500C26F4500B
:1011B8000822000E00220D500502F3500C26F450B0
:1011C8000822000E002202500402F3500826F450B0
:1011D800002202500502016A000E0122F350002687
:1011E800F45001220D500602F3500826F450002254
:1011F800026A000E012202220B500602F35000265A
:10120800F4500122000E02220E500602F35001266D
:10121800F450022202BE19EF09F0083600360136F2
:1012280002360306D8B43BEF09F02CEF09F0D8805A
:10123800800E08640030000E002201220222D8A08D
:101248002CEF09F0023201320032034A36EF09F07E
:101258000AAE029E000E3EEF09F0010E9EEC01F070
:101268003EEF09F0020EA5EC01F03EEF09F0040E86
:0612780091EC01F01200F0
:08127E00067E40EC03F01200B3
:10128600830EC2162AC300F0003600900036009086
:101296000050C212CAEC02F0C282C2A201D0FDD72F
:1012A600C4CF01F0006A00C02BF301C02CF3C35079
:1012B6000012000E011200C02BF301C02CF3000E29
:1012C6000014026E0150800B036E000E031802E13B
:1012D600000E021803E003012B6B2C6B2BC300F0EE
:0612E6002CC301F0120010
:1012EC0000C008F00150006E016A026A036A0B6AC2
:1012FC000C6A016A026A036A960E036E0A6A00AEF1
:10130C008EEF09F0081E001E082AD8B4002A0A8E97
:10131C0000C001F008C000F0086A026A50EC05F049
:02132C001200AD
:10132E000B6A0350D8B4DDEF09F002500A6E028E3C
:10133E008E0E035E03AEE1EF09F0036C080E035C44
:10134E00D8A0BCEF09F0036E013602C001F0026AAC
:10135E00080E035CD8A0BCEF09F0036E0136016ADB
:10136E000350D8A4D890C6EF09F00350D8B4C6EFF6
:10137E0009F0D89002320132032EC0EF09F00BBCF7
:10138E0001A0D3EF09F0D8A0D3EF09F0012AD8B409
:10139E00022A02BEF0EF09F00AAEF6EF09F0021EC5
:1013AE00011E012AD8B4022AF6EF09F0026A016A78
:1013BE00F6EF09F00B800BAEFAEF09F0026A0AAEF7
:1013CE00FAEF09F0FF0E026E016E0A360232FAEFE4
:1013DE0009F0010E0C6EBCEC02F0FCEF09F0000EF1
:1013EE000C6EFCEF09F0FF0E0C6E0150006E0250F9
:0413FE00016E12006A
:101402000134083609360450085E0550D8A0053C60
:10141200095E003601360F0E0C6E013408360936AD
:10142200045000A006D0085E0550D8A0053C095E15
:1014320005D008260550D8B0053C092600360136ED
:101442000C2EEBD700B006D0045008260550D8B0B9
:08145200053C09260000120010
:10145A002AC3E9FF2BC3EAFFEECF2CF3000E0301E8
:10146A002D6F000E2D6F000E2D1902E1200E2C1982
:10147A0007E0000E2D1902E1090E2C1901E003D034
:10148A002A4B2B2BE5D72E6B2F6B306B316B000E53
:10149A002D1902E12D0E2C1905E1304B312B2A4B67
:1014AA002B2B08D0000E2D1902E12B0E2C1902E16C
:1014BA002A4B2B2B2AC3E9FF2BC3EAFFEECF2CF3CF
:1014CA00000E2D6F000E2D6F2CC332F335DC005247
:1014DA0018E02EC300F02FC301F00A0E046E000EAE
:1014EA00056E02DC300E2C5D026E000E2D59036E65
:1014FA00025000242E6F035001202F6F2A4B2B2BF2
:10150A00D9D73051311108E02E510008006E2FC38F
:10151A0001F0000E015604D02EC300F02FC301F0D3
:02152A001200AD
:10152C00FC0EE96E000EEA6E03012A51E926D8B0D2
:10153C00EA2A2B51EE24326F3207EFEC02F0680EE0
:10154C000C6EE40E0D6E0D2EFED70C2EFCD700008B
:0A155C002CC332F389EC05F01200F5
:1015660003012E6B050E2E5D0AE22E512C25E16E2F
:10157600000E2D21E26E200EE66E2E2BF3D72E5195
:101586002C25E16E000E2D21E26EE66A2E072E5105
:101596002C252F6F000E2D21306F0A0E046E000EC3
:1015A600056E2AC300F02BC301F0D4EC02F008C08C
:1015B60000F009C001F0300E00262FC3E1FF30C352
:1015C600E2FF00C0E6FF0A0E046E000E056E2AC397
:1015D60000F02BC301F0D4EC02F000C02AF301C0E6
:1015E6002BF3000E011802E1000E001801E102D0F3
:0615F6002E07CDD7120004
:1015FC002AC3F6FF2BC3F7FF2CC3F8FF0900F5CF66
:10160C0001F001C02DF3010E03012A27000E2B233C
:10161C002C230150000A01E10CD02DC341F3B0EC96
:10162C0000F0850E0D6E0D2EFED703012D51000816
:04163C00DFE31200D6
:1016400043EC01F060C03BF3E0EC00F02AC33BF355
:10165000E0EC00F02BC33BF3E0EC00F0DEEC00F03C
:02166000120076
:1016620003012D6B2AC3E9FF2BC3EAFFEECF2CF354
:101672002C51000A0FE02CC341F3B0EC00F003013F
:101682002D2B2D512A25E96E000E2B21EA6EEECF6D
:061692002CF3EED712005C
:101698002AC3E9FF2BC3EAFFEE5003012C1905E129
:1016A8002AC300F02BC301F010D02AC300F02BC3CB
:1016B80001F02A4B2B2B00C0E9FF01C0EAFFEECF57
:0C16C80000F00052E5E1006A016A120027
:1016D4002AC302F02BC303F002C000F003C001F0E0
:1016E400024A032A00C0E9FF01C0EAFFEE5201E00A
:1016F400F3D703012A51025C006E2B510358016E8B
:0A170400010E005E000E015A1200F3
:10170E002EC300F003012E07005228E02AC3E9FF82
:10171E002BC3EAFFEE50000A0CE02AC3E9FF2BC3ED
:10172E00EAFF2CC3D9FF2DC3DAFFEE50DE1801E11C
:10173E000FD02AC3E9FF2BC3EAFF2CC3D9FF2DC359
:10174E00DAFFDE50EE5C006E016A000E015A08D020
:10175E0003012A4B2B2B2C4B2D2BD2D7006A016A5F
:02176E00120067
:1017700003012B6B2A5109081DE20A0E046E2AC3CD
:1017800000F06AEC06F000C02BF300C02BF32B37FF
:101790002B912B372B912B372B912B372B910A0E1B
:1017A000046E2AC300F06AEC06F008C000F0005096
:0E17B0002B1302D02AC32BF32BC300F0120020
:1017BE0043EC01F060C03BF3E0EC00F02AC33BF3D6
:1017CE00E0EC00F0D7EC05F0D10E03013B6FE0EC3E
:1017DE0000F00301326B04EC06F000C02BF3DEECDC
:0817EE0000F02BC300F0120013
:1017F6000B6A0C6A0A6A0350D8B445EF0CF0028EE5
:101806008E0E035E03BE0DEF0CF0D8B40DEF0CF098
:1018160049EF0CF0036C080E035CD8A024EF0CF023
:10182600036E013602C001F0026A080E035CD8A0FE
:1018360024EF0CF00136016A0350D8A4D8902EEF9D
:101846000CF00350D8B42EEF0CF0D89002320132CF
:10185600032E28EF0CF00BBC01A03BEF0CF0D8A038
:101866003BEF0CF0012AD8B4022A02BE58EF0CF066
:101876000AAE5EEF0CF0021E011E012AD8B4022A3F
:101886005EEF0CF0026A016A5EEF0CF00B800BAEA5
:1018960062EF0CF0026A0AAE62EF0CF0FF0E026E07
:1018A600016E0A36023262EF0CF0010E0C6EBCECD1
:1018B60002F064EF0CF0000E0C6E64EF0CF0FF0EFD
:0C18C6000C6E0150006E0250016E12000A
:1018D20013C300F0003600900036009000C0C2FF33
:1018E200C2809C0E0C6ED70E0D6E0D2EFED70C2EE6
:1018F200FCD7C28200000000C2A201D0FDD70000C6
:10190200C4CF01F0006AC3500026000E012212006B
:0E191200CF0E0D6E0D2EFED70000000012004D
:101920000050086E0150006E016A026A036A0B6A79
:101930000C6A960E036E0A6A00C001F008C000F03F
:0A194000086A026A50EC05F012007C
:10194A00020E0301136F000E146F176B186B9D9A2A
:10195A00FF0E02018C25E16E010E8D21E26EE66A10
:10196A00000E8D5D02E1150E8C5DD8B0CED0000E52
:10197A00006E8D51005C02E18C511208D8B0C5D0BE
:10198A00900E03012A6F620E2B6F000E2C6F31DE50
:10199A008CC22AF38DC22BF38E0E2C6F020E2D6F82
:1019AA00DDDD8E0E2A6F020E2B6F56DE52EC07F02B
:1019BA00020E0301156F000E166F02018D5103010D
:1019CA00165D04E102018C510301155D2EE2FF0E42
:1019DA001525E96E010E1621EA6EEE503B0A22E148
:1019EA00FF0E1525E16E010E1621E26EE66A830EE0
:1019FA001725196F020E18211A6FFF0E13252A6F69
:101A0A00010E14212B6F24DD19C3E1FF1AC3E2FF73
:101A1A0000C0E6FF010E1525136F000E1621146F84
:101A2A00174B182B154B162BC8D7830E1725196F72
:101A3A00020E18211A6FFF0E13252A6F010E1421A8
:101A4A002B6F06DD19C3E1FF1AC3E2FF00C0E6FFF0
:101A5A0083C281F284C282F285C2FCF286C2FBF2A0
:101A6A0087C2FAF288C2FDF20201FB5106080AE2B5
:101A7A00AF0E03012A6F5D0E2B6F000E2C6FB9DDBE
:101A8A000201FB6B03012A6B2B6BD5DDFDC22AF326
:101A9A006ADE00C02BF3010E2A6FCDDDFAC22AF3EB
:101AAA0062DE00C02BF3020E2A6FC5DDFBC22AF3E9
:101ABA005ADE00C02BF3030E2A6FBDDD81C22AF362
:101ACA0052DE00C02BF3040E2A6FB5DD82C22AF360
:101ADA004ADE00C02BF3050E2A6FADDDFCC22AF3E5
:101AEA0042DE00C02BF3060E2A6FA5DD070E0301A6
:101AFA002A6F100E2B6F9FDD380E03012A6F5E0EC0
:101B0A002B6F000E2C6F75DD0FD00301F80E2A6FB4
:101B1A005A0E2B6F000E2C6F6CDDD30E2A6F5D0EE2
:101B2A002B6F000E2C6F65DD050E0B6E0F0E0C6E03
:101B3A00F10E0D6E0D2EFED70C2EFCD70B2EFAD7FA
:101B4A000101FF6B0301176B186B016B026B02013A
:101B5A008C6B8D6BFE6BFF6BAECFF9F29D8A120018
:101B6A00000E0301141902E1000E131934E013C325
:101B7A00E9FF14C3EAFFEE522EE015C32AF316C397
:101B8A002BF3A3DD00C02EF313C32AF314C32BF3E4
:101B9A0015C32CF316C32DF3B5DD000E011802E1AF
:101BAA00000E001805E113C300F014C301F015D0AC
:101BBA00010E030113252A6F000E14212B6F15C382
:101BCA00E9FF16C3EAFFEECF2CF361DD00C013F381
:0C1BDA0001C014F3C5D7006A016A1200B4
:101BE60003011951000805E3070E1A6F000E1B6F5B
:101BF60012D01951160805E2170E1C6F000E1D6F44
:101C060006D01951010F1C6F1D6B000E1D231CC33E
:101C16001AF31DC31BF31AC324F31BC325F31E6B50
:101C26001F6B046A056A066A076A13C300F014C3C9
:101C360001F015C302F016C303F0ADEC06F0010E79
:101C4600D8B0000E006E005209E017C3E1FF18C3BA
:101C5600E2FF2D0EE66E174B182B157F13C304F00B
:101C660014C305F015C306F016C307F0006A016A2F
:101C7600026A036AADEC06F0010ED8B0000E006EE3
:101C8600005237E0000E046E000E056E000E066E62
:101C96007F0E076E13C300F014C301F015C302F0E4
:101CA60016C303F0ADEC06F0010ED8B0000E006EC0
:101CB60000521FE013C300F014C301F015C302F075
:101CC60016C303F0000E046E000E056E200E066E9F
:101CD600820E076EACEC08F000C013F301C014F3DB
:101CE60002C015F303C016F3010E1E5F000E1F5B44
:101CF600C9D7000E046E000E056E200E066E820E0B
:101D0600076E13C300F014C301F015C302F016C327
:101D160003F0ADEC06F0000ED8B0010E006E0052D6
:101D26001EE0000E046E000E056E200E066E820E7C
:101D3600076E13C300F014C301F015C302F016C3F7
:101D460003F0EEEC07F000C013F301C014F302C079
:101D560015F303C016F303011E4B1F2BCAD71E51E2
:101D660024271F512523010E206F000E216F000E20
:101D7600266F000E276F000E286F7F0E296F800ECC
:101D86002119006E800E2519005C02E12451205DA8
:101D96001EE2000E046E000E056E200E066E820E0A
:101DA600076E26C300F027C301F028C302F029C33B
:101DB60003F0EEEC07F000C026F301C027F302C0E3
:101DC60028F303C029F30301204B212BD8D7000E9B
:101DD600046E000E056E000E066E800E076E26C39C
:101DE60000F027C301F028C302F029C303F0EEEC8C
:101DF60007F013C304F014C305F015C306F016C3A9
:101E060007F040EC03F000C013F301C014F302C066
:101E160015F303C016F3000E046E000E056E200EB9
:101E2600066E820E076EADEC06F0000ED8B0010EFF
:101E3600006E00520BE0000E0301136F000E146FCC
:101E4600000E156F7F0E166F1E4B1F2B0301800EA3
:101E56001F19006E800E005C02E1000E1E5D38E266
:101E660017C3E1FF18C3E2FF300EE66E174B182BBF
:101E760017C3E1FF18C3E2FF2E0EE66E174B182BB1
:101E8600800E2519006E800E005C02E1000E245DB6
:101E960004E224511E5F25511F5BFF0E206FFF0ECB
:101EA600216F800E1F19006E800E2119005C02E161
:101EB60020511E5D0DE217C3E1FF18C3E2FF300E8D
:101EC600E66E174B182B010E205F000E215BE9D73B
:101ED600206B216B800E2119006E800E2519005C87
:101EE60002E12451205D63E213C300F014C301F044
:101EF60015C302F016C303F097EC09F000C022F3F5
:101F060001C023F3300E002617C3E1FF18C3E2FF1A
:101F160000C0E6FF174B182B21511F1902E11E5175
:101F2600201908E117C3E1FF18C3E2FF2E0EE66E83
:101F3600174B182B22C300F023C301F076EC09F0EF
:101F460000C026F301C027F302C028F303C029F31B
:101F560000C004F001C005F002C006F003C007F09F
:101F660013C300F014C301F015C302F016C303F047
:101F76003FEC09F000C013F301C014F302C015F3DF
:101F860003C016F3000E046E000E056E200E066EDC
:101F9600820E076EACEC08F000C013F301C014F318
:101FA60002C015F303C016F3204B212B93D717C39A
:0A1FB600E1FF18C3E2FFE66A120023
:101FC000F00E03011315006E008600C080F260C0A1
:101FD00038F3040E0010396FA2EC02F000C07FF25B
:101FE0000D0E0D6E0D2EFED760C038F3FB0E0201F4
:101FF00080150301396FA2EC02F000C07FF20D0ED4
:082000000D6E0D2EFED712003B
:10200800130E03012A6F600E2B6F000E2C6FFEEC6F
:102018000AF0010E136F000E146F800E1419006E73
:10202800800E005C02E1050E135D32E213C300F07E
:1020380014C301F00036009001364F0E0024E96EFB
:10204800000E0120EA6EEECF00F0EECF01F03C0E5C
:10205800046E000E056ED4EC02F000C02AF301C035
:102068002BF38E0E2C6F020E2D6FB3EC0AF0900E30
:102078002A6F020E2B6F31EC0BF0240E2A6F630EC1
:102088002B6F000E2C6FFEEC0AF0134B142BC5D7E8
:0620980052EC07F01200FB
:10209E0089880001656B666B636B646B5B6A5C6A57
:0220AE0012001E
:1020B000290E0B6E960E0C6E7F0E0D6E0D2EFED73A
:0A20C0000C2EFCD70B2EFAD71200ED
:1020CA00060E0C6E2B0E0D6E0D2EFED70C2EFCD7A7
:0220DA001200F2
:1020DC0003012A6BDFEC0BF000C0F0F2010E0301E0
:1020EC002A6FDFEC0BF000C0FDF2020E03012A6F29
:1020FC00DFEC0BF000C0FAF2030E03012A6FDFECE9
:10210C000BF000C0FBF2040E03012A6FDFEC0BF0A6
:10211C0000C081F2050E03012A6FDFEC0BF000C04A
:10212C0082F2060E03012A6FDFEC0BF000C0FCF20A
:10213C00FAC213F303011333139F1333139F133397
:10214C00139F1333139F030E2A6FB8EC0BF0005040
:10215C0013150101016F300E01270F0E0201FA1544
:10216C000101026F300E0227FDC213F3030113337A
:10217C00139F1333139F1333139F1333139F070EA4
:10218C002A6FB8EC0BF0005013150101046F300EE0
:10219C0004270F0E0201FD150101056F300E0527F6
:1021AC00F0C213F303011333139F1333139F133331
:1021BC00139F1333139F070E2A6FB8EC0BF00050CC
:1021CC0013150101076F300E07270F0E0201F015D2
:1021DC000101086F300E082781C213F3030113337A
:1021EC00139F1333139F1333139F1333139F070E34
:1021FC002A6FB8EC0BF00050131501010C6F300E68
:10220C000C270F0E0201811501010D6F300E0D27E9
:10221C0082C213F303011333139F1333139F13332E
:10222C00139F1333139F070E2A6FB8EC0BF000505B
:10223C00131501010F6F300E0F270F0E02018215BF
:10224C000101106F300E1027FCC213F3030113337E
:10225C00139F1333139F1333139F1333139F070EC3
:10226C002A6FB8EC0BF0005013150101126F300EF1
:10227C0012270F0E0201FC150101136F300E1327EC
:02228C0012003E
:10228E000301176B52EC07F0F2AE03D0010E0301FF
:10229E00176FF29EC190C296C294090E0B6E1E0E5F
:1022AE000C6EE40E0D6E03010D2EFDD70C2EFBD71A
:1022BE000B2EF9D70000156B166B136B146B800E7B
:1022CE001419006E800E005C02E1200E135D15E203
:1022DE002A6B43EC09F00050030115270150162319
:1022EE00D00E0C6EC90E0D6E0D2EFED70C2EFCD719
:1022FE0000000000134B142BE2D7050E006E15C321
:10230E0001F016C302F0005005E002320132029EC7
:10231E00FF0FFAD701C015F302C016F3010E025CCF
:10232E0002E1C20E015C07E31651020802E11551EB
:10233E00580801E320D00C0E2A6F5F0E2B6F000E93
:10234E002C6FFEEC0AF015C32AF316C32BF38E0E78
:10235E002C6F020E2D6FB3EC0AF08E0E2A6F020E4A
:10236E002B6F31EC0BF052EC07F0000E0001616F99
:10237E00020E626F62D015C361F016C362F0520E88
:10238E0003012A6F5C0E2B6F000E2C6FFEEC0AF011
:10239E0061C02AF362C02BF38E0E2C6F020E2D6FCE
:1023AE00B3EC0AF08E0E2A6F020E2B6F5DEC07F067
:1023BE008E0E2A6F020E2B6F31EC0BF0090E416F51
:1023CE00B0EC00F0EA0E03012A6F030E2B6F8EC2E3
:1023DE002CF314EC07F0D00E0C6EC90E0D6E0D2EF4
:1023EE00FED70C2EFCD700000000EB0E03012A6F67
:1023FE00030E2B6F8FC22CF314EC07F0D00E0C6E65
:10240E00C90E0D6E0D2EFED70C2EFCD7000000004F
:10241E00EC0E03012A6F030E2B6F90C22CF314ECFB
:10242E0007F0D00E0C6EC90E0D6E0D2EFED70C2EB3
:10243E00FCD70000000052EC07F003011751010A0F
:06244E00D8B4F28E12006A
:102454000301196B1A6B13C31BF314C31CF3800E13
:102464001419006E800E005C02E1000E135D0BE295
:10247400010E196F000E1A6F135100081B6F14C35D
:102484001CF3000E1C571BC32AF31CC32BF315C3E8
:102494002CF316C32DF3B3EC0AF0060E176F000EDF
:1024A400186F000E006E1851005C02E1175100080D
:1024B40019E217511525E16E18511621E26E010E2D
:1024C400175D006E000E1859016E00501525E96E57
:1024D40001501621EA6EEECFE6FF010E175F000EE3
:1024E400185BDFD715C3E1FF16C3E2FF200EE66ECB
:1024F40019511A111AE0176B186B17511525E96E4B
:1025040018511621EA6EEE50200A03E1174B182BDE
:10251400F4D7010E175F000E185B17511525E16EF5
:0C25240018511621E26E2D0EE66E12001A
:10253000400E0301326FEFEC02F00301156B080E41
:10254000155D13E2CF0E1525F66E620EF76E000EC6
:10255000F722000EF86E000EF8220900F5CF32F3D4
:1025600089EC05F00301152BEAD7020E326FEFEC70
:1025700002F013C32AF314C32BF303012C6B96EC64
:102580000AF0680E0C6EE40E0D6E0D2EFED70C2EAA
:06259000FCD70000120060
:10259600FC0EE96E000EEA6E03011351E926D8B06F
:1025A600EA2A1451EE24326F3207EFEC02F09C0E49
:1025B6000C6ED70E0D6E0D2EFED70C2EFCD715C346
:1025C6002AF316C32BF317C32CF335EC07F01200CE
:1025D60013C304F014C305F003011751181124E0C6
:1025E600010E175F000E185B04C002F005C003F071
:1025F600044A052A15C300F016C301F0154B162B25
:1026060000C0E9FF01C0EAFF02C0E1FF03C0E2FF2C
:10261600EECFE6FF02C0E9FF03C0EAFFEECF00F00F
:10262600005201E101D0D8D717C300F018C301F05A
:10263600010E175F000E185B0050011008E004C081
:10264600E1FF05C0E2FFE66A044A052AEDD713C397
:0826560000F014C301F01200B2
:10265E0013C304F014C305F004C002F005C003F068
:10266E00044A052A15C300F016C301F00301154BE9
:10267E00162B00C0E9FF01C0EAFF02C0E1FF03C054
:10268E00E2FFEECFE6FF02C0E9FF03C0EAFFEE5223
:0E269E0001E0E2D713C300F014C301F01200F4
:1026AC000301156B166B13C3E9FF14C3EAFFEE505D
:1026BC00000A17E0800E1619006E800E005C02E115
:1026CC00140E155D0EE213C3E9FF14C3EAFFEECF3F
:1026DC0032F389EC05F00301134B142B154B162B1D
:0426EC00E2D712001F
:1026F0000201E26BE36B94908B90020E0B6E040E62
:102700000C6EBA0E0D6E0D2EFED70C2EFCD70B2EB6
:10271000FAD700008B805D0E0D6E0D2EFED7E46B98
:10272000948000000000E26BE36B82B00AD0E24BC1
:10273000E32B010EE35D02E1900EE25D01E301D0C7
:10274000F4D7010EE35D02E1900EE25DD8A0E42B28
:10275000E26BE36B82A00AD0E24BE32B010EE35D58
:1027600002E1900EE25D01E301D0F4D7010EE35DDA
:1027700002E1900EE25DD8A0E42BE451020A6AE186
:102780008B82E06BE16B95EC07F000C0DEF295EC1C
:1027900007F000C0DFF295EC07F000C0ECF295EC1A
:1027A00007F000C0EDF295EC07F000C0EBF28B9261
:1027B000DF51DE25016E026A000E0222EC51012675
:1027C000000E0222ED510126000E0222FF0E01141E
:1027D000036E02C004F0000E0416000E041802E19D
:1027E000035000182EE1DEC2E5F2000EE66FE76F3F
:1027F000E86FE7C2E8F2E6C2E7F2E5C2E6F2E56BAF
:10280000DF51E513000EE613E713E813E7C2E8F221
:10281000E6C2E7F2E5C2E6F2E56BEC51E513000E25
:10282000E613E713E813E7C2E8F2E6C2E7F2E5C20F
:10283000E6F2E56BED51E513000EE613E713E8133E
:1028400008D0580EE56F580EE66F580EE76F580E19
:10285000E86F08D0630EE56F630EE66F630EE76FF7
:10286000630EE86F850E0D6E0D2EFED7E5C200F0EB
:0E287000E6C201F0E7C202F0E8C203F0120077
:10287E0015C3F6FF16C3F7FF17C3F8FF0900F5CF10
:10288E0000F0005218E015C3F6FF16C3F7FF17C38A
:10289E00F8FF0900F5CF00F013C3E1FF14C3E2FF08
:1028AE0000C0E6FF0301134B142B010E1527000E7B
:1028BE0016231723DDD713C3E1FF14C3E2FFE66A25
:0228CE001200F6
:1028D000800E03011419006E800E005C02E1000EF0
:1028E000135D08E213510008006E14C301F0000EDE
:0E28F000015604D013C300F014C301F012000F
:1028FE00A69C14C3AAFF13C3A9FFA69EA680A8CFA9
:04290E0000F01200C3
:102912000450000A08E10550000A05E1FF0E006EAE
:102922007F0E016E58D00D6A096A086A01500010C4
:10293200D8B4000C015005180A6E0ABE0D1E0B6AAF
:1029420005AE05D0041E051E042AD8B4052A01AE20
:1029520005D0001E011E002AD8B4012A015005101C
:102962000A6E0ABE10D001EC0AF00BB020D00DAEF8
:10297200000C001E011E002AD8B4012A081E091EDE
:10298200082AD8B4092A000C05AE0DD001BE07D022
:102992000150096E0050086E016A006AE8D7016AA8
:1029A200006A002A000C011E001E0B2ADDD7082A2D
:1029B200D8B4092A0450085CD8A4D9D70550095CB8
:1029C200D8A4D5D7096A086A002AD8B4012A01AE68
:0829D200CED70000FF0C12003B
:1029DA00620E03012A6F590E2B6F000E2C6FFEEC4C
:1029EA000AF0EA0E136F030E146F84DF00C034F18D
:1029FA00000E0101356F300E345D006E000E355940
:102A0A00016E640E046E000E056E79EC06F000C0CD
:102A1A0061F001C062F0EB0E0301136F030E146F35
:102A2A0069DF00C034F1000E0101356F300E345DEC
:102A3A00006E000E3559016E0A0E046E000E056E08
:102A4A0079EC06F000500001612701506223EC0E78
:102A5A000301136F030E146F4DDF00C034F1000E33
:102A6A000101356F300E345D006E000E3559016E6E
:102A7A00005000016125026E01506221036E02C0FE
:102A8A0061F003C062F0010E035C02E1C20E025C57
:102A9A0007E36251020802E161511C0801E30FD009
:102AAA00D00E03012A6F5E0E2B6F000E2C6FFEEC08
:102ABA000AF0000E0001616F020E626F1BD02C0E2D
:102ACA0003012A6F5B0E2B6F000E2C6FFEEC0AF0CF
:102ADA0061C02AF362C02BF38E0E2C6F020E2D6F8B
:102AEA00B3EC0AF08E0E2A6F020E2B6F31EC0BF04C
:062AFA0052EC07F012008F
:102B000005C307F306C308F307C313F308C314F39D
:102B1000F6DE00C009F3000E03010A6F000E0A1969
:102B200002E1000E091901E122D0800E030A006EB5
:102B3000800E0819005C02E10751FF0801E217D07E
:102B400009C341F3B0EC00F0340E0C6EF10E0D6EC3
:102B50000D2EFED70C2EFCD7000000000301074B02
:102B6000082B000E0A1902E1000E0919CDE112002E
:102B70000900F5CFE6FF0006FBE10106F9E11200CE
:102B8000A20E01013E6F010E3F6F000E406F000E5E
:102B9000416F860E4A6F020E4B6F000E4C6F000E97
:102BA0004D6FAE0E466F0B0E476F000E486F000E56
:102BB000496F080E656F0C0E666F320E676F030E5D
:102BC000686FC00E616F010E626F3B0E636F030E84
:102BD000646FBC0E6D6F010E6E6F000E6F6F000E96
:102BE000706F949894968B988B9694889486C79ED1
:082BF000C79C380EC66E1200EE
:102BF800600E0101696F010E6A6F410E6B6F030E63
:102C08006C6FE20E5D6F2F0E5E6F000E5F6F000E31
:102C1800606FFF0E546FFF0E556F000E566F000E5B
:102C2800576FFF0E506FFF0E516F000E526F000E60
:102C3800536FAC8A900EAB6E948E949C9EAA03D070
:082C4800AECF00F0FBD7120033
:102C5000660E046E660E056E660E066E820E076EBA
:102C600024C000F025C001F026C002F027C003F008
:102C7000ADEC06F0010ED8B0000E006E0052D8B4D4
:102C800085D1000E046E000E056E300E066E820EAB
:102C9000076E24C000F025C001F026C002F027C056
:102CA00003F0ADEC06F0000ED8B0010E006E00523D
:102CB000D8B46CD103010051010AD8A463D1046ACD
:102CC000056A066A076A6DC000F06EC001F06FC049
:102CD00002F070C003F0ADEC06F0000ED8B0010EAB
:102CE000006E0052D8B44ED124C004F025C005F0C7
:102CF00026C006F027C007F0CD0E006ECC0E016E88
:102D0000640E026E820E036E3FEC09F0FBEC0BF0DA
:102D100000C007F301C008F3150E2A6F630E2B6F76
:102D2000000E2C6FFEEC0AF007C32AF308C32BF346
:102D30008E0E2C6F020E2D6FB3EC0AF08E0E2A6FE2
:102D4000020E2B6F31EC0BF01D0E0725F66E630E95
:102D50000821F76E000EF86E000EF8220900F5CF7C
:102D600009F3000E0A6F09C300F00AC301F090ECEA
:102D70000CF000C00BF301C00CF302C00DF303C054
:102D80000EF3040E2A6F630E2B6F000E2C6FFEECF9
:102D90000AF009C32AF30AC32BF38E0E2C6F020E1E
:102DA0002D6FB3EC0AF08E0E2A6F020E2B6F31ECF2
:102DB0000BF00BC300F00CC301F00DC302F00EC307
:102DC00003F0330E046E330E056E330E066E7E0E68
:102DD000076EACEC08F0000E046E000E056E480E97
:102DE000066E850E076EEEEC07F000C00FF301C013
:102DF00010F302C011F303C012F300C013F301C0BB
:102E000014F302C015F303C016F38E0E0301176FFF
:102E1000020E186F030E196FF3EC0DF0E60E2A6F19
:102E20005F0E2B6F000E2C6FFEEC0AF08E0E2A6FD9
:102E3000020E2B6F31EC0BF0200E416FB0EC00F066
:102E40006DC004F06EC005F06FC006F070C007F0F2
:102E50000FC300F010C301F011C302F012C303F05E
:102E60003FEC09F0000E046E000E056E480E066E73
:102E7000850E076EACEC08F097EC09F000C005F386
:102E800001C006F30FC304F010C305F011C306F030
:102E900012C307F06DC000F06EC001F06FC002F009
:102EA00070C003F0ADEC06F0010ED8B0000E006E5D
:102EB000005217E003010551E808016E06C302F055
:102EC000030E025602500101185D02E10150175D28
:102ED00008E2030105510101172703010651010111
:102EE00018236DC004F06EC005F06FC006F070C00E
:102EF00007F00FC300F010C301F011C302F012C3BA
:102F000003F0ADEC06F0010ED8B0000E006E0052DA
:102F100014E005C313F306C314F3DADC01011851FE
:102F2000015C02E11751005C08E203010551010157
:102F3000172703010651010118230101010E17157E
:102F4000006E00B002D0BD9801D0BD8817C100F05E
:102F500018C101F001320032019E010E0014006E12
:102F600000B002D0BD9A01D0BD8A17C100F018C1CF
:102F700001F001320032019E01320032019E00C098
:102F8000BEFF03D00101176B186B19D09A0E030115
:102F90002A6F5F0E2B6F000E2C6FFEEC0AF0010102
:102FA000176B186B520E0B6E2B0E0C6E000E0D6E07
:102FB0000D2EFED70C2EFCD70B2EFAD700001200D8
:102FC00005C371F006C372F007C373F008C374F051
:102FD00009C342F10AC343F10BC344F10CC345F1E9
:022FE0001200DD
:102FE200AECF01F0ABA202D0AB98AB8801C000F02B
:022FF2001200CB
:102FF400D00E0001606F52EC07F0A40E03012A6F9B
:10300400610E2B6F000E2C6FFEEC0AF0290E0B6E76
:10301400960E0C6E7F0E0D6E0D2EFED70C2EFCD769
:103024000B2EFAD780BA57D0990E2A6F000E2B6F49
:1030340031EC0BF0020E0C6E080E0D6E0D2EFED749
:103044000C2EFCD700002A6B500E2B6F20EC0BF0DB
:10305400010E03012A6F300E2B6F20EC0BF00F0EC4
:1030640003012A6FB8EC0BF000C02BF3020E2A6F99
:1030740020EC0BF0030E03012A6F040E2B6F20ECDF
:103084000BF0040E03012A6F240E2B6F20EC0BF0BF
:10309400050E03012A6F080E2B6F20EC0BF0110EA6
:1030A40003012A6FB8EC0BF000C02BF3060E2A6F55
:1030B40020EC0BF0070E03012A6F100E2B6F20EC8F
:1030C4000BF0020E0C6E080E0D6E0D2EFED70C2E9C
:1030D400FCD7000009D0B40E03012A6F5F0E2B6FDA
:1030E400000E2C6FFEEC0AF06EEC10F0070E0201DD
:1030F400FB5D19E2030E006E000E016EFBC204F0CC
:10310400000E056E79EC06F0E70E0024E96E000E61
:103114000120EA6EEECF2AF3EECF2BF3EECF2CF3A1
:10312400FEEC0AF009D00301CE0E2A6F5F0E2B6F5E
:10313400000E2C6FFEEC0AF00C0E2A6F010E2B6FA2
:1031440031EC0BF0210E2A6F630E2B6F000E2C6FE7
:10315400FEEC0AF0010E2A6F010E2B6F31EC0BF01E
:0631640052EC07F012001E
:10316A0003010051010A43E1070E0201FB5D19E266
:10317A00030E006E000E016EFBC204F0000E056E17
:10318A0079EC06F0E70E0024E96E000E0120EA6EE3
:10319A00EECF2AF3EECF2BF3EECF2CF3FEEC0AF0B0
:1031AA0009D00301B80E2A6F610E2B6F000E2C6F27
:1031BA00FEEC0AF0210E2A6F630E2B6F000E2C6FA5
:1031CA00FEEC0AF00C0E2A6F010E2B6F31EC0BF09D
:1031DA003B0E416FB0EC00F0010E03012A6F010EA5
:1031EA002B6F31EC0BF03B0E416FB0EC00F012008C
:1031FA004E0E0001606F030E01010A15016E0BC12C
:10320A0002F0000E0216000E021802E1000E01186A
:10321A00D8A478D078EC13F000C0F5F201C0F6F229
:10322A0002C0F7F203C0F8F20350630A08E1025041
:10323A00630A05E10150630A02E10050630A0DE1E5
:10324A00040E0301136F010E146FE80E156F600E62
:10325A00166F000E176FCBEC12F00201F851580AE4
:10326A0008E1F751580A05E1F651580A02E1F55109
:10327A00580A0DE1040E0301136F010E146FD30EE9
:10328A00156F600E166F000E176FCBEC12F002016D
:10329A00F851630A08E1F751630A05E1F651630A36
:1032AA0002E1F551630A0DE0F851580A08E1F751B5
:1032BA00580A05E1F651580A02E1F551580A01E0A7
:1032CA0007D0EE6BEF6BF36BF46BE94BEA2B1AD07A
:1032DA00FF0EF515EE6FF651FF0BEF6FF7C200F018
:1032EA00F8C201F0026A036A00C0F5F201C0F6F200
:1032FA0002C0F7F203C0F8F2FF0E0014F36F015098
:10330A00FF0BF46F0201010EF115016EF2C202F019
:10331A00000E0216000E021802E1000E0118D8A4CF
:10332A002DD132C113F333C114F37F0E0301156F8C
:10333A00600E166F000E176F3FEC14F00201EF518A
:10334A00800802E1EE5100080FE2030E0101322566
:10335A00E16E000E3321E26E2D0EE66EFF0E0201C3
:10336A00EE177F0EEF1709D0030E01013225E16E29
:10337A00000E3321E26E200EE66E0101040E3225A4
:10338A000301056F000E010133210301066F640E6C
:10339A00046E000E056EEEC200F0EFC201F0D4EC2E
:1033AA0002F00A0E046E000E056ED4EC02F008C09C
:1033BA0000F009C001F0300E002605C3E1FF06C384
:1033CA00E2FF00C0E6FF050E010132250301056F89
:1033DA00000E010133210301066F0A0E046E000E6E
:1033EA00056EEEC200F0EFC201F0D4EC02F00A0E54
:1033FA00046E000E056ED4EC02F008C000F009C09D
:10340A0001F0300E002605C3E1FF06C3E2FF00C04B
:10341A00E6FF070E010132250301056F000E0101C7
:10342A0033210301066F0A0E046E000E056EEEC20A
:10343A0000F0EFC201F0D4EC02F008C000F009C0BD
:10344A0001F0300E002605C3E1FF06C3E2FF00C00B
:10345A00E6FF0201F451030802E1F351E8086CE3C4
:10346A000F0E010132250301056F000E0101332100
:10347A000301066F640E046E000E056EF3C200F0BF
:10348A00F4C201F0D4EC02F00A0E046E000E056ECE
:10349A00D4EC02F008C000F009C001F0300E00269A
:1034AA0005C3E1FF06C3E2FF00C0E6FF100E0101FB
:1034BA0032250301056F000E010133210301066F56
:1034CA000A0E046E000E056EF3C200F0F4C201F09B
:1034DA00D4EC02F00A0E046E000E056ED4EC02F073
:1034EA0008C000F009C001F0300E002605C3E1FF54
:1034FA0006C3E2FF00C0E6FF120E010132250301F6
:10350A00056F000E010133210301066F0A0E046ED6
:10351A00000E056EF3C200F0F4C201F0D4EC02F022
:10352A0008C000F009C001F0300E002605C3E1FF13
:10353A0006C3E2FF00C0E6FF0301D40E326FEFECD0
:10354A0002F032C113F333C114F356EC13F0040E34
:10355A00136F090E146F98EC12F01D0E0301136F0E
:10356A00010E146F32C115F333C116F32FEC13F0A9
:10357A00B00E0101256F3B0E276F3FD032C113F306
:10358A0033C114F3550E0301156F600E166F000E4A
:10359A00176F3FEC14F0010E010132250301136F7E
:1035AA00000E010133210301146F0C0E156F010E79
:1035BA00166F080E176F000E186FEBEC12F00A0E5A
:1035CA00010132250301136F000E010133210301AA
:1035DA00146F010E156F010E166F080E176F000E8D
:1035EA00186FEBEC12F0D40E326FEFEC02F032C12E
:0C35FA0013F333C114F356EC13F012006D
:10360600806A0F01386B388138833885EF0E926EE9
:1036160092988988928A396BFF0E816EFF0E936E9F
:10362600938293849388796A786A826A3A6BFF0EEA
:10363600946E94809492948494969488948E949C98
:0836460094928B92606A12005D
:10364E00FF0E0101156F010E166F15C1E9FF16C1B0
:10365E00EAFFEE50550A69E1130E1525E96E000ECC
:10366E001621EA6EEE50230A60E1160E03012A6F50
:10367E00620E2B6F000E2C6FFEEC0AF0FF0E2A6FFF
:10368E00010E2B6F31EC0BF052EC07F0D00E000157
:10369E00606FF29EA5EC0CF0300E0101015D006E24
:1036AE00016A000E015A580E046E020E056E79EC78
:1036BE0006F000C005F301C006F3300E025D006E89
:1036CE00016A000E015A3C0E046E000E056E79EC76
:1036DE0006F00050030105251E6E015006211F6ED7
:1036EE00300E0101045D006E016A000E015A0A0ED1
:1036FE00046E000E056E79EC06F000501E26015089
:10370E001F2205511E26000E1F22300E1E5E000EB9
:10371E001F5A4E0E0001606F01011B6B1C6B4FECAC
:10372E0010F00101156B166BF28EFF0E0301136F75
:10373E00010E146F410E156F000E166FB5EC0DF0E5
:10374E0000C015F101C016F1000E026E0150025CB0
:10375E0002E10050000854E2080E01011525E16E49
:10376E00000E1621E26EE66A060E152503012A6F7B
:10377E00000E0101162103012B6F2DEC0AF000C083
:10378E004DF001C04EF0000E026E0150025C02E1DF
:10379E0000501E0807E3000E4E5C02E1010E4D5C68
:1037AE0001E310D00301C70E2A6F620E2B6F000EBD
:1037BE002C6FFEEC0AF0050E4D6E000E4E6E4FECA9
:1037CE0010F01BD0F30E03012A6F610E2B6F000E4B
:1037DE002C6FFEEC0AF04DC02AF34EC02BF38E0E6A
:1037EE002C6F020E2D6FB3EC0AF08E0E2A6F020EA6
:1037FE002B6F31EC0BF052EC07F00101156B166BD1
:10380E00FF0E0301136F010E146F480E156F000E9D
:10381E00166FB5EC0DF000C015F101C016F1000EDB
:10382E00026E0150025C02E10050000813E2010E2C
:10383E0001011B6F000E1C6F610E03012A6F620ED9
:10384E002B6F000E2C6FFEEC0AF04FEC10F0010106
:10385E00156B166BFF0E0301136F010E146F3C0EEA
:10386E00156F000E166FB5EC0DF000C015F101C00E
:10387E0016F1000E026E0150025C02E100500008CB
:10388E0011E201011B6B1C6B6D0E03012A6F620EA0
:10389E002B6F000E2C6FFEEC0AF04FEC10F00101B6
:1038AE00156B166BFF0E0301136F010E146F2C0EAA
:1038BE00156F000E166FB5EC0DF000C015F101C0BE
:1038CE0016F1000E026E0150025C02E1005000087B
:1038DE0045E2040E01011525E96E000E1621EA6E71
:1038EE00EE50310A23E1000E1C1902E1000E1B19E5
:1038FE0014E18998010E0001656F000E666F450E8A
:10390E0003012A6F620E2B6F000E2C6FFEEC0AF075
:10391E001EC02AF01FC02BF009D00301940E2A6F8F
:10392E005E0E2B6F000E2C6FFEEC0AF0040E0101E2
:10393E001525E96E000E1621EA6EEE50300A0BE1E7
:10394E004FEC10F0360E03012A6F620E2B6F000E35
:10395E002C6FFEEC0AF00101156B166BFF0E0301C6
:10396E00136F010E146F350E156F000E166FB5EC3A
:10397E000DF000C015F101C016F1000E026E0150DF
:10398E00025C02E10050000833E2070E010115252A
:10399E00E96E000E1621EA6EEE50310A10E1010EAC
:1039AE001C6E000E1D6E760E03012A6F5E0E2B6FBF
:1039BE00000E2C6FFEEC0AF00101156B166B070E54
:1039CE001525E96E000E1621EA6EEE50300A10E152
:1039DE001C6A1D6A630E03012A6F5F0E2B6F000EA9
:1039EE002C6FFEEC0AF00101176B186B156B166B42
:1039FE00FF0E0301136F010E146F310E156F000EC3
:103A0E00166FB5EC0DF000C015F101C016F1000EE9
:103A1E00026E0150025C02E1005000083FE2040E0B
:103A2E0001011525E96E000E1621EA6EEE50310ADF
:103A3E001DE1000E1C1902E1010E1B190EE1010E13
:103A4E00206E000E216E7F0E03012A6F5F0E2B6F0C
:103A5E00000E2C6FFEEC0AF009D00301A80E2A6F9F
:103A6E005C0E2B6F000E2C6FFEEC0AF0040E0101A3
:103A7E001525E96E000E1621EA6EEE50300A0BE1A6
:103A8E00206A216A470E03012A6F5F0E2B6F000E0C
:103A9E002C6FFEEC0AF00101156B166BFF0E030185
:103AAE00136F010E146FC80E156F000E166FB5EC66
:103ABE000DF000C015F101C016F1000E026E01509E
:103ACE00025C02E10050000833E2080E01011525E8
:103ADE00E96E000E1621EA6EEE50310A11E1010E6A
:103AEE0000016B6F000E6C6F530E03012A6F620E96
:103AFE002B6F000E2C6FFEEC0AF00101156B166B8E
:103B0E00080E1525E96E000E1621EA6EEE50300AEB
:103B1E000CE1790E03012A6F620E2B6F000E2C6FD3
:103B2E00FEEC0AF000016B6B6C6B0101156B166BF2
:103B3E00FF0E0301136F010E146FC10E156F000EF1
:103B4E00166FB5EC0DF000C015F101C016F1000EA8
:103B5E00026E0150025C02E1005000081EE2B20E3D
:103B6E0003012A6F5E0E2B6F000E2C6FFEEC0AF017
:103B7E00E9C22AF3EAC22BF38E0E2C6F020E2D6FC2
:103B8E00B3EC0AF08E0E2A6F020E2B6F31EC0BF097
:103B9E0052EC07F00101156B166BFF0E0301136F4C
:103BAE00010E146FDB0E156F000E166FB5EC0DF0D7
:103BBE0000C015F101C016F1000E026E0150025C3C
:103BCE0002E10050000807E247EC11F052EC07F05A
:103BDE000101156B166BFF0E0301136F010E146FAF
:103BEE00D00E156F000E166FB5EC0DF000C015F16E
:103BFE0001C016F1000E026E0150025C02E100508F
:103C0E000008D8B038D2000E00016C1902E1010E86
:103C1E006B1902E104EC10F0010E0301326FEFECB0
:103C2E0002F0800E0301326FEFEC02F0020E0B6E0B
:103C3E00040E0C6EBA0E0D6E0D2EFED70C2EFCD78A
:103C4E000B2EFAD7000032C113F333C114F3510E09
:103C5E000301156F610E166F000E176F3FEC14F017
:103C6E003C0E046E000E056E51C000F052C001F005
:103C7E00D4EC02F000C034F101C035F10A0E01019E
:103C8E0032250301056F000E010133210301066F7A
:103C9E000A0E046E000E056ED4EC02F0300E0026F5
:103CAE0005C3E1FF06C3E2FF00C0E6FF0B0E0101F4
:103CBE0032250301056F000E010133210301066F4A
:103CCE000A0E046E000E056E34C100F035C101F00F
:103CDE00D4EC02F008C000F009C001F0300E00264E
:103CEE0005C3E1FF06C3E2FF00C0E6FF3C0E046E13
:103CFE00000E056E53C000F054C001F0D4EC02F07B
:103D0E0000C034F101C035F1110E0101322503015D
:103D1E00056F000E010133210301066F0A0E046EBA
:103D2E00000E056ED4EC02F0300E002605C3E1FF46
:103D3E0006C3E2FF00C0E6FF120E010132250301A9
:103D4E00056F000E010133210301066F0A0E046E8A
:103D5E00000E056E34C100F035C101F0D4EC02F056
:103D6E0008C000F009C001F0300E002605C3E1FFC7
:103D7E0006C3E2FF00C0E6FF32C113F333C114F3F2
:103D8E0056EC13F0C00E326FEFEC02F0020E0B6E1B
:103D9E00040E0C6EBA0E0D6E0D2EFED70C2EFCD729
:103DAE000B2EFAD7000032C113F333C114F3660E93
:103DBE000301156F610E166F000E176F3FEC14F0B6
:103DCE0051C02AF352C02BF38E0E03012C6F020E3C
:103DDE002D6FB3EC0AF0070E010132250301136FAC
:103DEE00000E010133210301146F8F0E156F020EA9
:103DFE00166F040E176F000E186FEBEC12F053C017
:103E0E002AF354C02BF38E0E2C6F020E2D6FB3ECD3
:103E1E000AF00E0E010132250301136F000E01018F
:103E2E0033210301146F8F0E156F020E166F040EE1
:103E3E00176F000E186FEBEC12F032C113F333C193
:103E4E0014F356EC13F0940E326FEFEC02F0020EF8
:103E5E000B6E040E0C6EBA0E0D6E0D2EFED70C2EC2
:103E6E00FCD70B2EFAD7000032C113F333C114F373
:103E7E003C0E0301156F610E166F000E176F3FECAF
:103E8E0014F03C0E046E000E056E55C000F056C0C8
:103E9E0001F0D4EC02F000C034F101C035F10A0E8D
:103EAE00010132250301056F000E010133210301CB
:103EBE00066F0A0E046E000E056ED4EC02F0300E84
:103ECE00002605C3E1FF06C3E2FF00C0E6FF0B0EAE
:103EDE00010132250301056F000E0101332103019B
:103EEE00066F0A0E046E000E056E34C100F035C169
:103EFE0001F0D4EC02F008C000F009C001F0300E61
:103F0E00002605C3E1FF06C3E2FF00C0E6FF3C0E3C
:103F1E00046E000E056E57C000F058C001F0D4ECD0
:103F2E0002F000C034F101C035F1110E010132254D
:103F3E000301056F000E010133210301066F0A0E06
:103F4E00046E000E056ED4EC02F0300E002605C392
:103F5E00E1FF06C3E2FF00C0E6FF120E01013225AB
:103F6E000301056F000E010133210301066F0A0ED6
:103F7E00046E000E056E34C100F035C101F0D4ECB4
:103F8E0002F008C000F009C001F0300E002605C393
:103F9E00E1FF06C3E2FF00C0E6FF32C113F333C1F7
:103FAE0014F356EC13F0D40E326FEFEC02F0020E57
:103FBE000B6E040E0C6EBA0E0D6E0D2EFED70C2E61
:103FCE00FCD70B2EFAD7000032C113F333C114F312
:103FDE00120E0301156F610E166F000E176F3FEC78
:103FEE0014F055C02AF356C02BF38E0E03012C6F1E
:103FFE00020E2D6FB3EC0AF0070E010132250301FC
:10400E00136F000E010133210301146F8F0E156F14
:10401E00020E166F040E176F000E186FEBEC12F0F7
:10402E0057C02AF358C02BF38E0E2C6F020E2D6F35
:10403E00B3EC0AF00F0E010132250301136F000ECF
:10404E00010133210301146F8F0E156F020E166FCF
:10405E00040E176F000E186FEBEC12F032C113F353
:10406E0033C114F356EC13F058EC10F058EC10F07A
:10407E000101156B166BFF0E0301136F010E146F0A
:10408E00BA0E156F000E166FB5EC0DF000C015F1DF
:10409E0001C016F1000E026E0150025C02E10050EA
:1040AE000008D8B02DD1060E01011527000E1623DB
:1040BE007D6B7E6B000E7E5D02E1040E7D5DD8B0E1
:1040CE0090D015C1E9FF16C1EAFF300EEE5C346FD9
:1040DE00356B000E355B15C1E9FF16C1EAFFEECF59
:1040EE0041F3B0EC00F034C100F035C101F00A0E1E
:1040FE00046E000E056E79EC06F000C034F101C0BE
:10410E0035F10101154B162B15C1E9FF16C1EAFF5A
:10411E00EECF41F3B0EC00F015C1D9FF16C1DAFFB6
:10412E00DE5001013427000E3523300E345F000EB1
:10413E00355B154B162B15C1E9FF16C1EAFFEECF05
:10414E0041F3B0EC00F00101154B162B000E006E82
:10415E003551005C02E1345104082DE2000E355D4C
:10416E0002E1170E345D27E2010E7D25036E000E6F
:10417E007E21046E03C000F004C001F000360090F2
:10418E000136710E00240301056F010E0120066F2A
:10419E0034C100F035C101F03C0E046E000E056E08
:1041AE0079EC06F005C3E1FF06C3E2FF00C0E6FFAF
:1041BE0001C0E6FF12D07DC100F07EC101F00036D5
:1041CE0000900136710E0024E16E010E0120E26EA8
:1041DE00E70EE66E030EE66E04D001017D4B7E2BDC
:1041EE0069D701017A51050802E17951280847E3A0
:1041FE007A51785D02E17951775D41E27851765DD1
:10420E0002E17751755D3BE27651745D02E17551C5
:10421E00735D35E2010E745D02E12C0E735D2FE3CA
:10422E00190E03012A6F5E0E2B6F000E2C6FFEEC23
:10423E000AF0010E01017D6F000E7E6F000E7E5D95
:10424E0002E1050E7D5D1AE27DC100F07EC101F036
:10425E000036009001364F0E0024E16E000E012054
:10426E00E26E710E0024E96E010E0120EA6EEECFB1
:10427E00E6FFEECFE6FF7D4B7E2BE0D73CD05F0E08
:10428E0003012A6F5B0E2B6F000E2C6FFEEC0AF0F3
:10429E00010E01017D6F000E7E6F000E7E5D02E14C
:1042AE00040E7D5D26E27DC100F07EC101F0003678
:1042BE0000900136710E0024E96E010E0120EA6EA7
:1042CE00EECF2AF3EECF2BF38E0E03012C6F020EE0
:1042DE002D6FB3EC0AF08E0E2A6F020E2B6F31EC9F
:1042EE000BF02E0E416FB0EC00F001017D4B7E2BDA
:1042FE00D4D752EC07F004EC10F00101156B166BDD
:10430E00FF0E0301136F010E146FB50E156F000E25
:10431E00166FB5EC0DF000C015F101C016F1000ED0
:10432E00026E0150025C02E10050000870E252EC95
:10433E0007F0570E03012A6F5E0E2B6F000E2C6FC7
:10434E00FEEC0AF0450E2A6F570E2B6F000E2C6FE7
:10435E00FEEC0AF0660E2A6F5D0E2B6F000E2C6FB0
:10436E00FEEC0AF0410E2A6F5D0E2B6F000E2C6FC5
:10437E00FEEC0AF0F60E2A6F5D0E2B6F000E2C6F00
:10438E00FEEC0AF0C30E2A6F5A0E2B6F000E2C6F26
:10439E00FEEC0AF08C0E2A6F5A0E2B6F000E2C6F4D
:1043AE00FEEC0AF0920E2A6F5B0E2B6F000E2C6F36
:1043BE00FEEC0AF08B0E2A6F5D0E2B6F000E2C6F2B
:1043CE00FEEC0AF0D10E2A6F5C0E2B6F000E2C6FD6
:1043DE00FEEC0AF0DF0E2A6F590E2B6F000E2C6FBB
:1043EE00FEEC0AF01B0E2A6F5A0E2B6F000E2C6F6E
:1043FE00FEEC0AF0210E2A6F590E2B6F000E2C6F59
:10440E00FEEC0AF052EC07F00101156B166B03017E
:10441E00016B026B000E025D02E17F0E015D12E286
:10442E00FF0E0125E16E010E0221E26EE66A010E1B
:10443E000125006E000E0221016E00C001F301C0C5
:10444E0002F3E8D7AECFF9F20101FF6B0201F96B6F
:10445E000301016B026B02018C6B8D6BFE6BFF6BAC
:04446E009D8A120011
:104472004E0E0001606F150E0B6E4B0E0C6EBE0ED3
:104482000D6E0D2EFED70C2EFCD70B2EFAD7000088
:10449200300E0301136FE0EC0FF0340E0C6EF10ED0
:1044A2000D6E0D2EFED70C2EFCD700000000300E34
:1044B2000301136FE0EC0FF0150E0C6EC60E0D6EBD
:1044C2000D2EFED70C2EFCD70000300E0301136F09
:1044D200E0EC0FF0150E0C6EC60E0D6E0D2EFED713
:1044E2000C2EFCD70000200E0301136FE0EC0FF03E
:1044F200150E0C6EC60E0D6E0D2EFED70C2EFCD7B1
:104502000000280E0301326FEFEC02F0150E0C6E64
:10451200C60E0D6E0D2EFED70C2EFCD70000080E17
:104522000301326FEFEC02F0150E0C6EC60E0D6E2B
:104532000D2EFED70C2EFCD70000010E0301326FA8
:10454200EFEC02F0050E0B6E0F0E0C6EF10E0D6EFF
:104552000D2EFED70C2EFCD70B2EFAD7060E03011A
:10456200326FEFEC02F0D00E0C6EC90E0D6E0D2EF6
:10457200FED70C2EFCD7000000000C0E0301326F98
:10458200EFEC02F0D00E0C6EC90E0D6E0D2EFED7A2
:0A4592000C2EFCD700000000120000
:10459C000B0ED76EDC0ED66E840ED56EF2945F6A5F
:0645AC00F28AF28E1200FB
:1045B2000301016B026B000E025D02E1800E015DE0
:1045C20012E2FF0E0125E16E010E0221E26EE66AA1
:1045D200010E0125006E000E0221016E00C001F3E2
:1045E20001C002F3E8D70101FF6B0301016B026B0B
:1045F2000101156B166B02018C6B8D6BFE6BFF6BF1
:0A460200AECFF9F2F96B9D8A1200A9
:10460C000301086B096B05C3F6FF06C3F7FF07C36D
:10461C00F8FF0900F5CF01F00150000A1DE0800EF3
:10462C000919006E800E005C02E1140E085D14E2A4
:10463C0005C3F6FF06C3F7FF07C3F8FF0900F5CF64
:10464C0032F389EC05F0010E03010527000E062359
:0A465C000723084B092BD7D71200E3
:1046660007C301F0010E006E015004E00036009011
:10467600FF0FFBD700C008F3001E05C3E9FF06C302
:10468600EAFF0050EF16120EE9260050EF1665EC11
:1046960010F003010851EF12120EE95E89EC0CF0DE
:1046A6000851EF14006F0051000A000ED8A4010E45
:0C46B600006F65EC10F000C300F0120073
:1046C200C26AC280C29CC29AC298C296C294C19E59
:1046D200C196C194C190C192C08EC092C084C09054
:0846E200C08AC088C0961200D6
:1046EA004E0E0001606F1D0E03012A6F010E2B6F23
:1046FA0031EC0BF03B0E416FB0EC00F05DC013F3F0
:10470A005EC014F38E0E0301156F020E166F2AECAB
:10471A0012F0000E00016C1902E1010E6B1913E18F
:10472A00090E03012A6F630E2B6F000E2C6FFEEC2D
:10473A000AF08F0E2A6F020E2B6F31EC0BF03B0E34
:10474A00416FB0EC00F0080E046E000E056E3AC11F
:10475A0000F03BC101F089EC14F000C05DF001C02B
:10476A005EF000016151005E6251015A00C03CF1E5
:10477A0001C03DF176EC09F0000E046E000E056EE4
:10478A00200E066E770E076EACEC08F000C06DF0D6
:10479A0001C06EF002C06FF003C070F0080E046E24
:1047AA00000E056E36C100F037C101F089EC14F035
:1047BA0000C069F001C06AF0000E00016C1902E144
:1047CA00000E6B190EE132C113F333C114F3290E33
:1047DA000301156F600E166F000E176F3FEC14F091
:1047EA000DD032C113F333C114F33F0E0301156F19
:1047FA00600E166F000E176F3FEC14F06DC013F3C6
:10480A006EC014F36FC015F370C016F38E0E030159
:10481A00176F020E186F020E196FF3EC0DF08E0E61
:10482A002A6F020E2B6F6AEC0BF000C034F101C044
:10483A0035F16DC004F06EC005F06FC006F070C0AF
:10484A0007F0006A016A026A036AADEC06F0010E1B
:10485A00D8B0000E006E00521DE0040E0101322590
:10486A00E16E000E3321E26E2B0EE66E050E322546
:10487A000301136F000E010133210301146F8E0E21
:10488A00156F020E166F34C117F335C118F3EBEC2E
:10489A0012F014D0040E010132250301136F000E29
:1048AA00010133210301146F8E0E156F020E166F6C
:1048BA0034C117F335C118F3EBEC12F0000E000106
:1048CA006C1902E1000E6B190CE1F1C22AF3F2C273
:1048DA002BF38E0E03012C6F020E2D6FB3EC0AF030
:1048EA000BD0030169C02AF36AC02BF38E0E2C6F1A
:1048FA00020E2D6FB3EC0AF00F0E010132250301EF
:10490A00136F000E010133210301146F8E0E156F10
:10491A00020E166F050E176F000E186FEBEC12F0F1
:10492A00800E326FEFEC02F032C113F333C114F38D
:10493A0056EC13F0090E01013225E16E000E332107
:10494A00E26E3B0EE66E000E00016C1902E1000EEB
:10495A006B1908E10A0E01013225E16E000E3321BE
:10496A00E26EE66A32C12AF333C12BF331EC0BF063
:10497A0002018E6B38C100F039C101F001320032F8
:10498A00019E01320032019E01320032019E00C0B6
:10499A0067F001C068F000C02AF301C02BF38E0E45
:1049AA0003012C6F020E2D6FB3EC0AF067C000F002
:1049BA0068C001F090EC0CF0330E046E330E056EF5
:1049CA00730E066E770E076EACEC08F0000E046EDE
:1049DA00000E056E700E066E810E076E40EC03F037
:1049EA0000C024F001C025F002C026F003C027F061
:1049FA00000E00016C1902E1010E6B1913E1110E90
:104A0A0003012A6F630E2B6F000E2C6FFEEC0AF067
:104A1A008F0E2A6F020E2B6F31EC0BF03B0E416F9B
:104A2A00B0EC00F019C100F01AC101F001320032F5
:104A3A00019E01320032019E01320032019E00C005
:104A4A0022F001C023F000C02AF301C02BF38E0E1E
:104A5A0003012C6F020E2D6FB3EC0AF0000E000159
:104A6A006C1902E1010E6B1913E10D0E03012A6F95
:104A7A00630E2B6F000E2C6FFEEC0AF08F0E2A6F5E
:104A8A00020E2B6F31EC0BF03B0E416FB0EC00F0D5
:104A9A0032C113F333C114F3FD0E0301156F5F0E18
:104AAA00166F000E176F3FEC14F0090E0101322544
:104ABA00E16E000E3321E26E300E2824006E00C033
:104ACA00E6FF0F0E3225E16E000E3321E26E300E44
:104ADA002024006E00C0E6FFC00E0301326FEFEC27
:104AEA0002F032C113F333C114F356EC13F032C19E
:104AFA0013F333C114F3270E156F610E166F000EF0
:104B0A00176F3FEC14F01EC02AF31FC02BF38E0E52
:104B1A0003012C6F020E2D6FB3EC0AF0040E010193
:104B2A0032250301136F000E010133210301146FB3
:104B3A008E0E156F020E166F050E176F000E186F88
:104B4A00EBEC12F024C013F325C014F326C015F3BE
:104B5A0027C016F38E0E176F020E186F020E196F0A
:104B6A00F3EC0DF08E0E2A6F020E2B6F6AEC0BF02F
:104B7A0000C034F101C035F10E0E010132250301E6
:104B8A00136F000E010133210301146F8E0E156F8E
:104B9A00020E166F00C017F301C018F3EBEC12F007
:104BAA00940E326FEFEC02F032C113F333C114F3F7
:104BBA0056EC13F0090E01013225E16E000E332185
:104BCA00E26E3B0EE66E000E00016C1902E1010E68
:104BDA006B1907E132C12AF333C12BF331EC0BF025
:104BEA0012D0000E1D1802E1010E1C180CE10A0E6B
:104BFA000101322503012A6F000E0101332103014D
:104C0A002B6F31EC0BF0030132C113F333C114F3F0
:104C1A00260E156F620E166F000E176F3FEC14F01A
:104C2A0017C113F318C114F38E0E0301156F020E88
:104C3A00166F2AEC12F00201956B93C294F22E0EB3
:104C4A00936F000E0101185D02E10A0E175D03E27F
:104C5A00300E0201926F080E010132250301136F13
:104C6A00000E010133210301146F8F0E156F020E1E
:104C7A00166F060E176F000E186FEBEC12F0000E8F
:104C8A001D1802E1010E1C1806E132C12AF333C1D4
:0C4C9A002BF331EC0BF052EC07F0120091
:104CA600F70E03012A6F5C0E2B6F000E2C6FFEECC5
:104CB6000AF094840F01496BFF0EBB6E0C0EBD6E9D
:104CC600BE6A060EBA6E94940101176B186BBD98F6
:104CD60017C100F018C101F001320032019E010E29
:104CE6000014006E00B002D0BD9A01D0BD8A17C173
:104CF60000F018C101F001320032019E013200328B
:084D0600019E00C0BEFF120077
:104D0E00FC0E03010525E96E000E0621EA6EEECFBC
:104D1E0032F3EFEC02F07B0E03012A6F610E2B6F64
:104D2E00000E2C6F35EC07F0FC0E03010525E96E25
:104D3E00000E0621EA6EEECF32F3EFEC02F0120017
:104D4E00C190C296C2940301136B69EC0CF000C0C3
:104D5E005DF001C05EF0005001013A2701503B2387
:104D6E00C286D00E0C6EC90E0D6E0D2EFED70C2EF9
:104D7E00FCD700000000020E0301136F69EC0CF06B
:104D8E0000C069F001C06AF00050010136270150E1
:104D9E003723030E0301136F69EC0CF000C022F0F1
:104DAE0001C023F000500101192701501A23C296A9
:104DBE00C284C180D00E0C6EC90E0D6E0D2EFED7A4
:104DCE000C2EFCD70000000002018E6B010E0301B9
:104DDE00136F69EC0CF000C067F001C068F0005072
:0A4DEE00010138270150392312009B
:104DF80094EC31F0D38CD38AD398D392D3909B8CF4
:104E080003EC1BF001017D6B7E6B000E7E5D02E101
:104E1800800E7D5D0AE2FF0E7D25E16E010E7E218A
:104E2800E26EE66A7D4B7E2BF0D77D6B7E6B000EC3
:104E38007E5D02E1500E7D5D0AE28E0E7D25E16EFB
:104E4800020E7E21E26EE66A7D4B7E2BF0D77D6BEB
:104E58007E6B000E7E5D02E1800E7D5D0AE27F0EB4
:104E68007D25E16E010E7E21E26EE66A7D4B7E2B8A
:104E7800F0D77D6B7E6B7F0E326F010E336F1C6A2D
:104E88001D6A00016B6B6C6B0201E06BE16B00014A
:104E9800E56BE66B0201E96BEA6B01011B6B1C6BAE
:104EA8004FEC10F0286A296A206A216AB886010E38
:104EB800B06EA00EAF6EAC84FCEC15F00C0E0301C6
:104EC800416FB0EC00F058EC10F052EC07F0E00E37
:104ED80003012A6F610E2B6F000E2C6FFEEC0AF097
:104EE800010E01017D6F000E7E6F000E7E5D02E1F6
:104EF8000B0E7D5D1CE2030E006E000E016E7DC17F
:104F080004F07EC105F079EC06F0750E0024E96E18
:104F1800000E0120EA6EEECF2AF3EECF2BF3EECF90
:104F28002CF3FEEC0AF001017D4B7E2BDED7F20E4E
:104F380003012A6F620E2B6F000E2C6FFEEC0AF035
:104F4800056B066B80EC15F058EC10F052EC07F08E
:104F5800EDEC14F0CC0E03012A6F610E2B6F000EDE
:104F68002C6FFEEC0AF0500EC86EC0EC15F0DEECAB
:104F780000F0E80E0301056F030E066F000E076FC1
:104F8800086F6E0E096F010E0A6F410E0B6F030E4C
:104F98000C6FE0EC17F0FAEC17F0000E246E000E20
:104FA800256E400E266E820E276E79DE58EC10F0C4
:104FB8004E0E0001606F39EC22F0010E0301326FD2
:104FC800EFEC02F032C113F333C114F32A0E0301DC
:104FD800156F5F0E166F000E176F3FEC14F0C00EC2
:104FE8000301326FEFEC02F0020E0B6E040E0C6E32
:104FF800BA0E0D6E0D2EFED70C2EFCD70B2EFAD73F
:10500800000032C12AF333C12BF36AEC0BF000C065
:1050180034F101C035F1000E026E0150025C02E16C
:10502800005014080CE2140E010132250301136F1D
:10503800000E010133210301146F56EC13F0800EAA
:10504800326FEFEC02F0020E0B6E040E0C6EBA0E0D
:105058000D6E0D2EFED70C2EFCD70B2EFAD70000A6
:10506800010134513225E16E35513321E26EE66A91
:1050780032C113F333C114F356EC13F0940E326FAC
:10508800EFEC02F0020E0B6E040E0C6EBA0E0D6EF3
:105098000D2EFED70C2EFCD70B2EFAD70000050ECE
:1050A8000301056F620E066F000E076F06EC23F012
:1050B80058EC10F058EC10F07F0E0101326F010E21
:1050C800336F010E0301326FEFEC02F0800E030123
:1050D800326FEFEC02F0020E0B6E040E0C6EBA0E7D
:1050E8000D6E0D2EFED70C2EFCD70B2EFAD7000016
:1050F800BE0E0301056F600E066F000E076F06EC0B
:1051080023F0C00E326FEFEC02F0020E0B6E040EAD
:105118000C6EBA0E0D6E0D2EFED70C2EFCD70B2E74
:10512800FAD70000A90E0301056F600E066F000E86
:10513800076F06EC23F0940E326FEFEC02F0020ECC
:105148000B6E040E0C6EBA0E0D6E0D2EFED70C2EC5
:10515800FCD70B2EFAD70000940E0301056F600EE2
:10516800066F000E076F06EC23F0D40E326FEFECDB
:1051780002F0020E0B6E040E0C6EBA0E0D6E0D2EA2
:10518800FED70C2EFCD70B2EFAD70000FD0E03011C
:10519800056F600E066F000E076F06EC23F058ECE3
:1051A80010F058EC10F0F292F288F19CF28EF60EA4
:1051B8002A6F5B0E2B6F000E2C6FFEEC0AF061EC71
:1051C80023F0170E2A6F580E2B6F000E2C6FFEEC73
:1051D8000AF09E0E2A6F580E2B6F000E2C6FFEECF5
:1051E8000AF052EC07F0010E01010A6F000E0B6F76
:1051F800F28CF28E030E0301056F000E066F83DD3D
:10520800030E0301136F010E146F6A0E156F600E03
:10521800166F000E176FCBEC12F0040E0301056F2A
:10522800000E066F70DD820E0301056F0F0E066F0C
:10523800076B33EC23F00201F16BF26B010E0101F5
:105248000A6F000E0B6F3A6B3B6B386B396B366B22
:10525800376B196B1A6B77DDD00E0001606F6EEC3F
:1052680010F0300E015D006E016A000E015A580EF2
:10527800046E020E056E79EC06F000C003F301C05F
:1052880004F3300E025D006E016A000E015A3C0EF6
:10529800046E000E056E79EC06F00050030103253C
:1052A8001E6E015004211F6E300E0101045D006E58
:1052B800016A000E015A0A0E046E000E056E79ECA2
:1052C80006F000501E2601501F2205511E26000E12
:1052D8001F22300E1E5E000E1F5A4E0E0001606F18
:1052E800D9EC22F001010B51000802E10A5107082C
:1052F800D8B08CD16BC000F3B5EC18F052501F5CDD
:1053080002E151501E5C07E354501F5C02E1535008
:105318001E5C01E20ED056501F5C02E155501E5C27
:1053280007E358501F5C02E157501E5C01E201D0B0
:1053380005D0010E286E000E296E02D0286A296A4F
:10534800020E0201F45D02E1580EF35D09E2000E5F
:10535800006E2950005C02E12850000801E210D0DC
:10536800000E211802E1010E201809E1000E006E5E
:105378002950005C02E12850000801E201D082D0E7
:10538800020E286E000E296E000E0001661902E159
:10539800000E651916E1000E01011C1902E1010E4B
:1053A8001B190FE1000E5C1802E1000E5B1809E101
:1053B800010E0001656F000E666F1EC02AF01FC047
:1053C8002BF050501F5C02E14F501E5C13E352500B
:1053D8001F5C02E151501E5C0DE21F50545C02E15B
:1053E8001E50535C07E256501F5C02E155501E5C8C
:1053F80001E20ED01F50585C02E11E50575C07E2D4
:105408005A501F5C02E159501E5C01E201D00AD0DB
:10541800000E006E5C50005C02E15B50000802E286
:105428005B6A5C6A0001000E661902E1010E6519EB
:1054380029E14D502A24016E4E502B20026E01C0E6
:105448004EF102C04FF102501F5C02E101501E5C98
:1054580014E28998010E656F000E666F1E500101F7
:105468004E5D0001636F1F5001014F590001646FC9
:10547800010E5B6E000E5C6E05D0656B666B8988ED
:10548800636B646B8E0E0301136F020E146F850E2F
:10549800156F620E166F000E176F3FEC14F0300E8A
:1054A80028240201966F8E0E03012A6F020E2B6FBD
:1054B80031EC0BF0000E01011C1902E1010E1B1961
:1054C8000AE1BF0E03012A6F620E2B6F000E2C6FCC
:1054D800FEEC0AF009D00301B70E2A6F620E2B6F9B
:1054E800000E2C6FFEEC0AF0000E0001661902E1B6
:1054F800010E65190AE1E50E03012A6F620E2B6F92
:10550800000E2C6FFEEC0AF009D00301D70E2A6FAB
:10551800620E2B6F000E2C6FFEEC0AF063C013F3C3
:1055280064C014F38E0E156F020E166F2AEC12F07B
:10553800190E2A6F630E2B6F000E2C6FFEEC0AF00B
:10554800910E2A6F020E2B6F31EC0BF03B0E416F60
:10555800B0EC00F0330E046E330E056E630E066E6B
:10556800820E076E24C000F025C001F026C002F0AC
:1055780027C003F0ADEC06F0010ED8B0000E006EA7
:1055880000520EE01CC000F328EC16F0030E0301D5
:105598002A6F0D0E2B6F3D0E2C6F96EC0AF01ED065
:1055A800000E1D1802E1010E1C1809E11C0E030172
:1055B8002A6F5D0E2B6F000E2C6FFEEC0AF00301B4
:1055C8001C6A1D6A006B28EC16F0030E03012A6F93
:1055D8000D0E2B6F480E2C6F96EC0AF0FDEC18F0B0
:1055E80075EC23F00201F14BF22B010E01010A6F59
:1055F800000E0B6F196B1A6B366B376B386B396B88
:105608003A6B3B6B0201E06BE16B03D001010A4B83
:105618000B2BCEEC22F0000E0201FF1902E1000E66
:10562800FE1904E15F50000A01E1F5D7000EFF19E9
:1056380002E1010EFE1902E127EC1BF00CD6FFD7A0
:1063280010EE1CF0430E006E010E016E5B0EF66E51
:10633800580EF76E000EF86EB8EC15F010EE61F01E
:10634800540E006E010E016EA80EF66E560EF76E14
:10635800000EF86EB8EC15F010EE5FF0010E006E4E
:10636800010E016E060EF66E000EF76E000EF86E48
:10637800B8EC15F010EEB5F0600E006E010E016E6F
:10638800480EF66E560EF76E000EF86EB8EC15F065
:026398001200F1
:0100060000F9
:0556480048656C7000D4
:07564D00506C6167653D0030
:0756540053746174757300CB
:08565B00566572626F73650071
:0B56630053686F7720506C6167650092
:0A566E005A65726F5F416D707300A2
:02567800000030
:10567A00AE6200FE6200F862009B6200EC6200A566
:05568A006200DE620079
:05568F000080C094D46E
:0956940030303A30303A30300079
:02569D0000000B
:09569F0030302F30302F30300084
:0256A800000000
:0256AA000000FE
:0256AC000000FC
:0256AE000000FA
:0256B0000000F8
:0256B2000100F5
:0456B40000000000F2
:0456B80000000000EE
:1056BC007B6100D25700906100E05800EE5E00550F
:1056CC005A00255C00C45B008C5700A15900FC56A5
:0456DC00007D5C00F1
:1056E000696E69742052544320445331333037205B
:0C56F000706172206465666175742000B2
:1056FC00204454483232204D65732E252048756D58
:10570C0069646974652065742054656D702E416DF3
:10571C00622E2028696E74657276616C6C65203E11
:10572C003173656320657420542E4F2E3D323575D0
:09573C00532F626974200D0A006C
:105745003C5A65726F5F416D70733E206661697486
:1057550020756E207A65726F20636170746575724D
:105765002041435337313220657420736175766566
:10577500206C276F666665737420656E20454570DD
:07578500726F6D0D0A200098
:10578C00205574696C6973652054696E795F525445
:10579C00435F4453313330372E632C4448543232F8
:1057AC005F414D323330325F53656E736F722E63CF
:1057BC00206574205F4C63645F347832305F49320B
:0657CC00432E630D0A00EC
:1057D200204469726563746F7279203A433A5C5F60
:1057E2004D696B726F435C5F4D657350726F6A6592
:1057F20074735F4D696B726F435C5F497272696764
:105802006174696F6E5F536F6C61725F73797374E9
:05581200656D0D0A00A8
:105817002054657374205520426174746572792031
:1058270028302D313556204D7573742062652073ED
:1058370063616C656420746F20322C3520746F208F
:1058470035562C206F6E2045413120696E70757476
:04585700200D0A0016
:02585B0000004B
:02585D00000049
:02585F00000047
:02586100000045
:04586300000040827F
:0258670000003F
:0258690000003D
:05586B005070652000F3
:04587000414146006C
:0758740043686172676500E3
:05587B004D616E750097
:07588000447572656520000C
:055887004175746F0083
:02588C00050015
:0C588E0000006801A4017404B004A0052F
:02589A0000000C
:02589C0000000A
:10589E002046696C746572696E6720414443206DC1
:1058AE006561737572652062792061726974686DC5
:1058BE00657469632061766572616765206F662025
:1058CE00415645524147455F76616C756573200DB3
:0258DE000A00BE
:1058E0002050726F6A6574203A31384632364B3236
:1058F000325F49727269676174696F6E5F554152B8
:10590000545F4144435F525443313330375F44481E
:105910005432325F323031382E6D637070690D0A47
:015920000086
:105921003C553B32383B30353B31383B30313B31F4
:10593100333B3533233E204D69736520E0204A6FA8
:10594100757220525443203238206D616920323003
:105951003138204C756E64692031334835330D0A76
:015961000045
:10596200205A65726F205368696674206F66204101
:1059720043533731322072656D6F766564206279E8
:10598200204F50455241544F5220646563697369F8
:0F5992006F6E202875736520425029200D0A0082
:1059A1002053414E532043617074657572205365D5
:1059B1006368657265737365206176656320466F00
:1059C1007572636865205358204C4D333933202E4E
:0E59D1002E2052454D4F56454420210D0A0010
:1059DF003C506C6167653D30373B30383B31383B6D
:1059EF0031393E20706C61676520686F7261697232
:1059FF006520646520374820612038482065742071
:0C5A0F003138482061203139480D0A0070
:105A1B003C53686F7720506C6167653E206166660A
:105A2B0069636861676520706C6167657320686F77
:105A3B0072616972657320656E20636F7572732076
:0A5A4B00737572204C43440D0A00ED
:105A550020436F6E66696720626974203A20313889
:105A65004632364B32325F466F73635F696E7465DB
:105A7500726E655F3878345F33324D487A2E6366CF
:075A8500677363680D0A005E
:105A8C003C4175746F3E202043646520506F6D70EF
:105A9C006520656E20666F6E6374696F6E20646539
:105AAC007320706172616D657472657320696D70BD
:075ABC006F73E9730D0A008E
:105AC3003C50706520303E20206F7520312C2050D3
:105AD3006F6D7065204F4646206F75204F4E20280E
:105AE300656E206D616E75207365756C656D656E91
:055AF30074290D0A00FA
:105AF8000D0A2052617070656C20666F726D61745A
:105B080020646520636465203A2022553B32343B8B
:105B180030383B31373B30343B31373B3336232247
:045B2800200D0A0042
:105B2C0020526563757065726174696F6E20416D8A
:105B3C007073204F666673657420656E2045455002
:105B4C00524F4D203078303345412C422C43203A73
:035B5C000D0A002F
:105B5F002E2E4572726F72203A2072616E67652029
:105B6F00203548204C6F77204C696D6974202E2E9C
:105B7F00203232482048696768204C696D6974206B
:035B8F000D0A00FC
:105B92003C44757265652078783E2044757265656F
:105BA200206D617263686520706F6D70652061762B
:105BB200656320787820303120E02032354D6E0D3B
:025BC2000A00D7
:105BC40020536F75726365203A205F313846323650
:105BD4004B32325F49727269676174696F6E5F43F9
:105BE4006F6E74726F6C5F3138303532382E630DDE
:025BF4000A00A5
:105BF600204D795F496E69745F41444320706F752B
:105C060072204541302C4541312C45413320657485
:0F5C1600204541323D20567265662D200D0A0053
:105C250020456570726F6D3A205F31384632364BCC
:105C350032325F49727269676174696F6E5F436F73
:0D5C45006E74726F6C2E696865780D0A0030
:105C52002053746F726520416D7073204F666673B6
:105C6200657420746F20454550524F4D2030783076
:0B5C72003345412C422C43203A200017
:105C7D00204D6F64756C65204843303620706F750C
:105C8D007220426C7565546F6F7468204170706C32
:0B5C9D0069636174696F6E200D0A00DE
:105CA8000D0A436465204172726F7361676520460F
:105CB8006F72636520656E204155544F207365757A
:095CC8006C656D656E740D0A0037
:105CD1003C43686172676520313E20206F7520303A
:105CE1002C20313D4368617267652062617474657F
:065CF1007269650D0A0056
:105CF70020496E742050574D3120313062697473DA
:105D07002061742031303030487A206F6E20524342
:055D170032200D0A001E
:105D1C000D0A42617474657269652043686172672B
:105D2C00E96520212053544F5020636861726765E8
:055D3C0075720D0A0064
:105D41003C41414620303E206F7520312C2041726C
:105D5100726F7361676520204155544F20464F5241
:055D610043450D0A009E
:105D66003C5374617475733E204574617420434FCF
:105D76004D206475206361707465757220445448C3
:055D860032320D0A009D
:105D8B003C566572626F736520313E206F75203013
:105D9B002C20313D42617661726420303D4D75653A
:045DAB00740D0A0069
:105DAF000D0A45727265757220456372697475725A
:105DBF0065206A6F75722053656D61696E65206A23
:045DCF00530D0A0066
:105DD30020706F757220323420416F757420323019
:105DE3003137204A657564692031374833360D0AE7
:035DF3000D0A0096
:105DF6003C4D616E753E202043646520506F6D708A
:105E06006520656E206D6F6465204D616E75656CED
:035E16000D0A0072
:105E19000D0A4E6F7576656C6C6520706C616765EF
:0F5E290020486F7261697265203A20200D0A00CF
:105E38000D0A45637269747572652064616E73201A
:0F5E48004453313330372E2E2E204F4B0D0A008E
:105E57003C48656C703E203A4C69737465206465F4
:0F5E67007320636F6D6D616E646573200D0A00AB
:105E76000D0A4D69736520456E204368617267653A
:0E5E860020426174746572792E2E2E0D0A0072
:105E94000D0A4364652050706520656E204D414EA7
:0E5EA40055207365756C656D656E740D0A0092
:105EB2000D0A20537461747573203A204E62204497
:0E5EC20065666175742044544832323D2000FC
:105ED0002042696720446F756274206F6E20414DC7
:0E5EE0005053204F666673657420210D0A0032
:105EEE002049727269676174696F6E20436F6E74B8
:0E5EFE00726F6C2053797374656D200D0A006D
:105F0C005042202120436865636B205A65726F20D4
:0E5F1C00416D7073202C2066756E64203A0073
:105F2A005F31384632364B32325F49727269676185
:0D5F3A0074696F6E5F436F6E74726F6C0060
:105F47000D0A4172726F73616765204155544F2086
:0C5F5700464F524345204F46460D0A00BD
:105F63000D0A41727265742043686172676520424D
:0C5F73006174746572792E2E2E0D0A00E8
:105F7F000D0A4172726F73616765204155544F204E
:0B5F8F00464F524345204F4E0D0A00C4
:105F9A000D0A2050726F626C656D652073757220F0
:0A5FAA0055626174202E2E0D0A00CE
:105FB4002052652D4C6563747572652052544320DC
:0A5FC4004453313330372020200011
:105FCE0020457272657572204A6F75722053656D29
:085FDE0061696E6521202000BD
:105FE600202043616C63756C617465645F49436826
:075FF600617267653D2000A8
:105FFD004175746F72697A3D2020204141463D20E4
:06600D00202020202000ED
:10601300506C6167657320486F72616972657320A4
:066023003A20200D0A00E6
:10602900416D703D202020202020496E643D2020B4
:06603900202020202000C1
:10603F00416D703D2020202020204541323D202001
:06604F00202020202000AB
:10605500202020202020202020202020202020203B
:056065002020202000B6
:10606A00204448543232206D65737572652054207D
:05607A00262048200073
:10607F0054703D2020202E2020432048753D2020A5
:05608F00202E20250079
:10609400496E697420525443204F4B202020202005
:0560A400202020200077
:1060A90050574D312C4F57532C49324320445331CB
:0560B900333037200028
:1060BE0031384632364B32322033324D487A204D0B
:0560CE0043372E3200F3
:1060D300445448323220436865636B2073756D20E6
:0560E3004572722E0061
:1060E8004454483232204E6F20726573706F6E735D
:0560F8006520202000DE
:1060FD00496E6974204144432041302C41312C417B
:05610D00322C413300BB
:1061120020496E64203D20202E2E2E2E2061202E1E
:056122002E2E2E2000CE
:10612700544D6E3D20202020202055423D20202028
:056137002020205600AD
:10613C00536F69722020646520202E2E4820612028
:05614C00202E2E48008A
:106151004D6174696E20646520202E2E48206120D7
:05616100202E2E480075
:1061660020496E64203D20202E2E2E2E2061202ECA
:056176002E2E2E20007A
:10617B002020202020202020202020202020202014
:05618B0020202020008F
:10619000204D696B726F432070726F20372E323042
:0461A000200A0D00C4
:1061A40020496E69742052544320445331333037AC
:0461B400200D0A00B0
:1061B800457272657572204A6F75722053656D61FC
:0461C800696E650097
:1061CC0020496E697420493243203130304B687A53
:0461DC00200D0A0088
:1061E0002050726573656E746174696F6E203A2019
:0361F0000D0A0095
:1061F3000D0A4F4B202C4E65772064757265653D03
:02620300200079
:1062050056657273696F6E203A20313830353238F1
:016215000088
:106216000D0A52544320557064617465203A20007B
:106226003B49526174696F3D203130302E30250074
:0F6236000D0A507065204F4646204F4B0D0A0051
:0E6245000D0A507065204F4E204F4B0D0A0081
:0E6253000D0A426176617264204F4B0D0A0005
:0C6261000D0A4175746F204F4B0D0A00B0
:0C626D000D0A4D616E75204F4B0D0A00AC
:0C6279000D0A4D756574204F4B0D0A0096
:0B6285004175746F72697A3D203B0088
:0B62900020496E64657831203D20003D
:0A629B004D657263726564692E00A0
:0962A50056656E647265646900BF
:0962AE0044696D616E63686500CE
:0862B7004D6F64653D303B00B2
:0862BF004D6F64653D313B00A9
:0862C7000D0A4241440D0A00DA
:0862CF000E0A0E0000000000A1
:0762D7005070653D303B00F3
:0762DE0053616D6564690066
:0762E5005070653D313B00E4
:0662EC004A6575646900BB
:0662F200202843292000D2
:0662F8004D6172646900B3
:0662FE004C756E6469009E
:05630400204B3D2000CC
:0463090045303D00DE
:04630D0045333D00D7
:0463110045313D00D5
:046315004D3D2000DA
:0463190041723D0090
:04631D000F324B648C
:0363210020200039
:03632400483B00F3
:020000040030CA
:0D000100381E3CFFBF81FF0FC00FE00F4015
:0200000400F00A
:10000000002D0000000000000000000000000000C3
:100010007061756C666A756A6F30300000000000B0
:1000200000000000000000000000000000000000D0
:1000300000000000000000000000000000000000C0
:1000400000000000000000000000000000000000B0
:1000500000000000000000000000000000000000A0
:00000001FF
